:020000040800F2
:1000000000000524E5200008E11C0008E31C0008AE
:10001000E51C0008E71C0008E91C000800000000BF
:10002000000000000000000000000000EB1C0008C1
:10003000ED1C000800000000EF1C0008F11C000887
:100040003521000835210008352100083521000838
:100050003521000835210008352100083521000828
:10006000352100083521000835210008F91C000859
:100070003521000835210008352100083521000808
:10008000352100083521000835210008091D000828
:1000900035210008191D0008352100083521000808
:1000A00035210008352100083521000835210008D8
:1000B00035210008291D0008391D000835210008D8
:1000C00035210008352100083521000835210008B8
:1000D00035210008491D0008352100083521000898
:1000E00035210008352100080000000035210008F6
:1000F0003521000835210008352100083521000888
:100100003521000835210008352100083521000877
:100110003521000835210008352100083521000867
:100120003521000835210008352100083521000857
:10013000352100083521000835210008591D000827
:1001400000000000000000000000000000000000AF
:100150003521000835210008352100083521000827
:100160003521000835210008352100083521000817
:100170003521000835210008352100080000000065
:1001800035210008352100083521000835210008F7
:1001900035210008352100083521000835210008E7
:1001A0003521000835210008352100080000000035
:1001B00035210008352100083521000835210008C7
:1001C0003521000835210008000000000000000073
:1001D00000000000000000003521000800000000C1
:1001E000000000000000000000000000000000000F
:1001F0000000000000000000352100083521000843
:1002000035210008352100080000000035210008D4
:100210003521000835210008352100083521000866
:100220003521000800000000352100080000000012
:1002300035210008352100080000000035210008A4
:100240003521000835210008352100083521000836
:100250003521000835210008352100083521000826
:100260003521000835210008352100083521000816
:100270003521000835210008352100080000000064
:1002800035210008352100083521000835210008F6
:1002900000000000352100083521000800000000A2
:1002A0000000000035210008352100083521000834
:1002B00035210008352100083521000835210008C6
:0C02C00035210008352100083521000818
:1002D00010B5054C237833B9044B13B10448AFF380
:1002E00000800123237010BD58040024000000008A
:1002F0006CB5000808B5034B1BB103490348AFF3C5
:10030000008008BD000000005C0400246CB50008FB
:1003100081F0004102E000BF83F0004330B54FEAB6
:1003200041044FEA430594EA050F08BF90EA020F23
:100330001FBF54EA000C55EA020C7FEA645C7FEAB6
:10034000655C00F0E2804FEA5454D4EB5555B8BFD9
:100350006D420CDD2C4480EA020281EA030382EA4A
:10036000000083EA010180EA020281EA0303362DDC
:1003700088BF30BD11F0004F4FEA01314FF4801CAF
:100380004CEA113102D0404261EB410113F0004FC1
:100390004FEA03334CEA133302D0524263EB430378
:1003A00094EA050F00F0A780A4F10104D5F1200E16
:1003B0000DDB02FA0EFC22FA05F2801841F1000171
:1003C00003FA0EF2801843FA05F359410EE0A5F145
:1003D00020050EF1200E012A03FA0EFC28BF4CF076
:1003E000020C43FA05F3C01851EBE37101F000452C
:1003F00007D54FF0000EDCF1000C7EEB00006EEB39
:100400000101B1F5801F1BD3B1F5001F0CD34908C2
:100410005FEA30004FEA3C0C04F101044FEA445219
:1004200012F5800F80F09A80BCF1004F08BF5FEAA0
:10043000500C50F1000041EB045141EA050130BD80
:100440005FEA4C0C404141EB0101013C28BFB1F592
:10045000801FE9D291F0000F04BF01460020B1FADD
:1004600081F308BF2033A3F10B03B3F120020CDAB0
:100470000C3208DD02F1140CC2F10C0201FA0CF08E
:1004800021FA02F10CE002F11402D8BFC2F1200CF3
:1004900001FA02F120FA0CFCDCBF41EA0C019040A9
:1004A000E41AA2BF01EB0451294330BD6FEA0404F2
:1004B0001F3C1CDA0C340EDC04F11404C4F12002DD
:1004C00020FA04F001FA02F340EA030021FA04F3EF
:1004D00045EA030130BDC4F10C04C4F1200220FA46
:1004E00002F001FA04F340EA0300294630BD21FA84
:1004F00004F0294630BD94F0000F83F4801306BF4A
:1005000081F480110134013D4EE77FEA645C18BF3D
:100510007FEA655C29D094EA050F08BF90EA020FD4
:1005200005D054EA000C04BF1946104630BD91EACC
:10053000030F1EBF0021002030BD5FEA545C05D1CF
:100540004000494128BF41F0004130BD14F580040E
:100550003CBF01F5801130BD01F0004545F0FE4182
:1005600041F470014FF0000030BD7FEA645C1ABFB7
:10057000194610467FEA655C1CBF0B46024650EAEE
:10058000013406BF52EA033591EA030F41F400211A
:1005900030BD00BF90F0000F04BF0021704730B5A0
:1005A0004FF4806404F132044FF000054FF0000175
:1005B00050E700BF90F0000F04BF0021704730B536
:1005C0004FF4806404F1320410F0004548BF40420B
:1005D0004FF000013EE700BF42004FEAE2014FEA60
:1005E00031014FEA02701FBF12F07F4393F07F4F3B
:1005F00081F06051704732F07F4208BF704793F03E
:100600007F4F04BF41F40021704730B54FF4607450
:1006100001F0004521F000411CE700BF50EA010253
:1006200008BF704730B54FF000050AE050EA0102FC
:1006300008BF704730B511F0004502D5404261EB6C
:1006400041014FF4806404F132045FEA915C3FF4AD
:10065000D8AE4FF003025FEADC0C18BF03325FEA4A
:10066000DC0C18BF033202EBDC02C2F1200300FAFB
:1006700003FC20FA02F001FA03FE40EA0E0021FA20
:1006800002F11444BDE600BF70B54FF0FF0C4CF40E
:10069000E06C1CEA11541DBF1CEA135594EA0C0FC0
:1006A00095EA0C0F00F0DEF82C4481EA030621EAFB
:1006B0004C5123EA4C5350EA013518BF52EA033536
:1006C00041F4801143F4801338D0A0FB02CE4FF0E8
:1006D0000005E1FB02E506F00042E0FB03E54FF018
:1006E0000006E1FB03569CF0000F18BF4EF0010E10
:1006F000A4F1FF04B6F5007F64F5407404D25FEA0C
:100700004E0E6D4146EB060642EAC62141EA5551BE
:100710004FEAC52040EA5E504FEACE2EB4F1FD0C00
:1007200088BFBCF5E06F1ED8BEF1004F08BF5FEA7E
:10073000500E50F1000041EB045170BD06F0004630
:1007400046EA010140EA020081EA0301B4EB5C04DD
:10075000C2BFD4EB0C0541EA045170BD41F48011D5
:100760004FF0000E013C00F3AB8014F1360FDEBFFA
:10077000002001F0004170BDC4F10004203C35DAD6
:100780000C341BDC04F11404C4F1200500FA05F359
:1007900020FA04F001FA05F240EA020001F00042FA
:1007A00021F0004110EBD37021FA04F642EB060170
:1007B0005EEA430E08BF20EAD37070BDC4F10C049A
:1007C000C4F1200500FA04F320FA05F001FA04F25E
:1007D00040EA020001F0004110EBD37041F100014A
:1007E0005EEA430E08BF20EAD37070BDC4F1200555
:1007F00000FA05F24EEA020E20FA04F301FA05F2BD
:1008000043EA020321FA04F001F0004121FA04F264
:1008100020EA020000EBD3705EEA430E08BF20EA34
:10082000D37070BD94F0000F0FD101F0004640006E
:1008300041EB010111F4801F08BF013CF7D041EAF0
:10084000060195F0000F18BF704703F000465200F4
:1008500043EB030313F4801F08BF013DF7D043EAC5
:100860000603704794EA0C0F0CEA135518BF95EA7B
:100870000C0F0CD050EA410618BF52EA4306D1D102
:1008800081EA030101F000414FF0000070BD50EA21
:10089000410606BF1046194652EA430619D094EAAB
:1008A0000C0F02D150EA013613D195EA0C0F05D195
:1008B00052EA03361CBF104619460AD181EA0301E9
:1008C00001F0004141F0FE4141F470014FF00000A1
:1008D00070BD41F0FE4141F4780170BD70B54FF03C
:1008E000FF0C4CF4E06C1CEA11541DBF1CEA1355BC
:1008F00094EA0C0F95EA0C0F00F0A7F8A4EB05049E
:1009000081EA030E52EA03354FEA013100F0888094
:100910004FEA03334FF0805545EA131343EA12635D
:100920004FEA022245EA111545EA10654FEA002612
:100930000EF000419D4208BF964244F1FD0404F5CB
:10094000407402D25B084FEA3202B61A65EB030527
:100950005B084FEA32024FF480104FF4002CB6EBE4
:10096000020E75EB030E22BFB61A754640EA0C0064
:100970005B084FEA3202B6EB020E75EB030E22BFA4
:10098000B61A754640EA5C005B084FEA3202B6EBE5
:10099000020E75EB030E22BFB61A754640EA9C00A4
:1009A0005B084FEA3202B6EB020E75EB030E22BF74
:1009B000B61A754640EADC0055EA060E18D04FEA32
:1009C000051545EA16754FEA06164FEAC30343EAD2
:1009D00052734FEAC2025FEA1C1CC0D111F4801F9F
:1009E0000BD141EA00014FF000004FF0004CB6E798
:1009F00011F4801F04BF01430020B4F1FD0C88BF37
:100A0000BCF5E06F3FF6AFAEB5EB030C04BFB6EB41
:100A1000020C5FEA500C50F1000041EB045170BD34
:100A20000EF0004E4EEA113114EB5C04C2BFD4EB61
:100A30000C0541EA045170BD41F480114FF0000EE5
:100A4000013C90E645EA060E8DE60CEA135594EA61
:100A50000C0F08BF95EA0C0F3FF43BAF94EA0C0F64
:100A60000AD150EA01347FF434AF95EA0C0F7FF4D9
:100A700025AF104619462CE795EA0C0F06D152EA2D
:100A800003353FF4FDAE1046194622E750EA410611
:100A900018BF52EA43067FF4C5AE50EA41047FF422
:100AA0000DAF52EA43057FF4EBAE12E74FF0FF3C87
:100AB00006E000BF4FF0010C02E000BF4FF0010C58
:100AC0004DF804CD4FEA410C7FEA6C5C4FEA430CD1
:100AD00018BF7FEA6C5C1BD001B050EA410C0CBF20
:100AE00052EA430C91EA030F02BF90EA020F002082
:100AF000704710F1000F91EA030F58BF994208BFE9
:100B000090422CBFD8176FEAE37040F001007047A5
:100B10004FEA410C7FEA6C5C02D150EA013C07D1FC
:100B20004FEA430C7FEA6C5CD6D152EA033CD3D047
:100B30005DF8040B704700BF8446104662468C4641
:100B40001946634600E000BF01B5FFF7B7FF002874
:100B500048BF10F1000F01BD4DF808EDFFF7F4FF9D
:100B60000CBF012000205DF808FB00BF4DF808ED28
:100B7000FFF7EAFF34BF012000205DF808FB00BF4B
:100B80004DF808EDFFF7E0FF94BF012000205DF86D
:100B900008FB00BF4DF808EDFFF7CEFF94BF012022
:100BA00000205DF808FB00BF4DF808EDFFF7C4FF1B
:100BB00034BF012000205DF808FB00BF4FEA41026E
:100BC000B2F1E04324BFB3F5001CDCF1FE5C0DD9AB
:100BD00001F0004C4FEAC0024CEA5070B2F1004FF5
:100BE00040EB830008BF20F00100704711F0804FF8
:100BF00021D113F13872BCBF01F00040704741F4BD
:100C000080114FEA5252C2F11802C2F1200C10FAC0
:100C10000CF320FA02F018BF40F001004FEAC123A4
:100C20004FEAD32303FA0CFC40EA0C0023FA02F348
:100C30004FEA4303CCE77FEA625307D150EA01331E
:100C40001EBF4FF0FE4040F44000704701F00040EE
:100C500040F0FE4040F40000704700BF80F00040CC
:100C600002E000BF81F0004142001FBF5FEA410384
:100C700092EA030F7FEA226C7FEA236C6AD04FEA84
:100C80001262D2EB1363C1BFD218414048404140C9
:100C9000B8BF5B42192B88BF704710F0004F40F47B
:100CA000000020F07F4018BF404211F0004F41F497
:100CB000000121F07F4118BF494292EA030F3FD063
:100CC000A2F1010241FA03FC10EB0C00C3F1200376
:100CD00001FA03F100F0004302D5494260EB400005
:100CE000B0F5000F13D3B0F1807F06D340084FEA70
:100CF000310102F10102FE2A51D2B1F1004F40EB65
:100D0000C25008BF20F0010040EA030070474900CC
:100D100040EB0000013A28BFB0F5000FEDD2B0FA69
:100D200080FCACF1080CB2EB0C0200FA0CF0AABF8C
:100D300000EBC25052421843BCBFD040184370472A
:100D400092F0000F81F4000106BF80F40000013230
:100D5000013BB5E74FEA41037FEA226C18BF7FEA07
:100D6000236C21D092EA030F04D092F0000F08BF49
:100D70000846704790EA010F1CBF0020704712F030
:100D80007F4F04D1400028BF40F00040704712F16F
:100D900000723CBF00F50000704700F0004343F0D4
:100DA000FE4040F4000070477FEA226216BF08460A
:100DB0007FEA23630146420206BF5FEA412390EACD
:100DC000010F40F4800070474FF0000304E000BFC3
:100DD00010F0004348BF40425FEA000C08BF704774
:100DE00043F0964301464FF000001CE050EA010238
:100DF00008BF70474FF000030AE000BF50EA01024D
:100E000008BF704711F0004302D5404261EB410139
:100E10005FEA010C02BF84460146002043F0B6435E
:100E200008BFA3F18053A3F50003BCFA8CF2083A83
:100E3000A3EBC25310DB01FA02FC634400FA02FC8C
:100E4000C2F12002BCF1004F20FA02F243EB020093
:100E500008BF20F00100704702F1200201FA02FCF5
:100E6000C2F1200250EA4C0021FA02F243EB0200E8
:100E700008BF20EADC7070474FF0FF0C1CEAD0522C
:100E80001EBF1CEAD15392EA0C0F93EA0C0F6FD0ED
:100E90001A4480EA010C400218BF5FEA41211ED0CB
:100EA0004FF0006343EA501043EA5111A0FB0131B7
:100EB0000CF00040B1F5000F3EBF490041EAD3718C
:100EC0005B0040EA010062F17F02FD2A1DD8B3F108
:100ED000004F40EBC25008BF20F00100704790F077
:100EE000000F0CF0004C08BF49024CEA502040EAC9
:100EF00051207F3AC2BFD2F1FF0340EAC25070478F
:100F000040F400004FF00003013A5DDC12F1190FCC
:100F1000DCBF00F000407047C2F10002410021FA3E
:100F200002F1C2F1200200FA02FC5FEA310040F156
:100F3000000053EA4C0308BF20EADC70704792F0CF
:100F4000000F00F0004C02BF400010F4000F013A07
:100F5000F9D040EA0C0093F0000F01F0004C02BF02
:100F6000490011F4000F013BF9D041EA0C018FE771
:100F70000CEAD15392EA0C0F18BF93EA0C0F0AD077
:100F800030F0004C18BF31F0004CD8D180EA01009D
:100F900000F00040704790F0000F17BF90F0004F36
:100FA000084691F0000F91F0004F14D092EA0C0F18
:100FB00001D142020FD193EA0C0F03D14B0218BFAB
:100FC000084608D180EA010000F0004040F0FE40F1
:100FD00040F40000704740F0FE4040F4400070478D
:100FE0004FF0FF0C1CEAD0521EBF1CEAD15392EA0C
:100FF0000C0F93EA0C0F69D0A2EB030280EA010CFC
:1010000049024FEA402037D04FF0805343EA111194
:1010100043EA10130CF000408B4238BF5B0042F1F2
:101020007D024FF4000C8B4224BF5B1A40EA0C0097
:10103000B3EB510F24BFA3EB510340EA5C00B3EBC9
:10104000910F24BFA3EB910340EA9C00B3EBD10FB7
:1010500024BFA3EBD10340EADC001B0118BF5FEA09
:101060001C1CE0D1FD2A3FF650AF8B4240EBC25032
:1010700008BF20F0010070470CF0004C4CEA5020F3
:101080007F32C2BFD2F1FF0340EAC250704740F442
:1010900000004FF00003013A37E792F0000F00F034
:1010A000004C02BF400010F4000F013AF9D040EAB2
:1010B0000C0093F0000F01F0004C02BF490011F446
:1010C000000F013BF9D041EA0C0195E70CEAD1533E
:1010D00092EA0C0F08D142027FF47DAF93EA0C0F25
:1010E0007FF470AF084676E793EA0C0F04D14B0209
:1010F0003FF44CAF08466EE730F0004C18BF31F0BB
:10110000004CCAD130F000427FF45CAF31F00043B4
:101110007FF43CAF5FE700BF4FEA4002B2F1FE4F01
:101120000FD34FF09E03B3EB12620DD94FEA0023A9
:1011300043F0004310F0004F23FA02F018BF404282
:1011400070474FF00000704712F1610F01D1420269
:1011500005D110F0004008BF6FF0004070474FF01D
:101160000000704742000ED2B2F1FE4F0BD34FF099
:101170009E03B3EB126209D44FEA002343F000430D
:1011800023FA02F070474FF00000704712F1610F30
:1011900001D1420202D14FF0FF3070474FF0000002
:1011A000704700BF53B94AB9002908BF00281CBFC7
:1011B0004FF0FF314FF0FF3000F06CB9ADF1080C8B
:1011C0006DE904CE00F006F8DDF804E0DDE9022365
:1011D00004B070472DE9F047089E0D4604468E4640
:1011E000002B40F082808A42174646D9B2FA82F23A
:1011F0004AB1C2F1200105FA02F320FA01F1974049
:1012000041EA030E94404FEA1748230CBEFBF8FC5A
:10121000B9B208FB1CEE43EA0E430CFB01F0984206
:101220000AD9FB180CF1FF3580F01681984240F284
:101230001381ACF1020C3B441B1AA4B2B3FBF8F0CF
:1012400008FB103344EA034400FB01F1A14209D931
:101250003C1900F1FF3380F00181A14240F2FE8091
:1012600002383C44641A40EA0C4000211EB1D440CC
:101270000023C6E90043BDE8F08702B9FFDEB2FAF9
:1012800082F2002A4FD1CB1B4FEA174E1FFA87F884
:101290000121B3FBFEFC250C0EFB1C3345EA034584
:1012A00008FB0CF3AB4207D97D190CF1FF3002D2D9
:1012B000AB4200F2E7808446ED1AA3B2B5FBFEF024
:1012C0000EFB105543EA054408FB00F8A04507D97A
:1012D0003C1900F1FF3302D2A04500F2D780184636
:1012E000A4EB080440EA0C40C0E78B4208D9002E6A
:1012F00000F0AF800021C6E900050846BDE8F08790
:10130000B3FA83F100294BD1AB4202D3824200F2FF
:10131000B780841A65EB030301209E46002EAAD0F5
:10132000C6E9004EA7E7C2F1200C01FA02F397408C
:1013300020FA0CF04FEA174E21FA0CFC1843BCFBC4
:10134000FEF1050C0EFB11CC1FFA87F845EA0C459F
:1013500001FB08F3AB4204FA02F409D97D1901F14B
:10136000FF3C80F08B80AB4240F2888002393D44E4
:10137000EB1A85B2B3FBFEF00EFB103345EA0345D2
:1013800000FB08F3AB4207D97D1900F1FF3C71D295
:10139000AB426FD902383D44EB1A40EA014178E78D
:1013A000C1F1200C8B4022FA0CF71F4320FA0CF4F9
:1013B00005FA01F34FEA174E25FA0CF51C43230CEE
:1013C000B5FBFEF91FFA87F80EFB195543EA0545F0
:1013D00009FB08FAAA4502FA01F200FA01F308D95A
:1013E0007D1909F1FF3047D2AA4545D9A9F1020973
:1013F0003D44A5EB0A05A4B2B5FBFEF00EFB10556B
:1014000044EA054400FB08F8A04507D93C1900F15F
:10141000FF352DD2A0452BD902383C4440EA094083
:10142000A4EB0804A0FB02894C45C6464D4619D3DF
:1014300016D05EB1B3EB0E0264EB050404FA0CFCAB
:10144000CA404CEA0202CC40C6E900240021BDE8B3
:10145000F087314630460EE7AC46EDE6184601E728
:101460004345E6D2B8EB020E69EB07050138E0E729
:101470002846D3E760468FE78146BAE7614677E7BB
:1014800008464BE7ACF1020C3D4415E702383C44FA
:1014900026E700BF704700BF844641EA000313F00F
:1014A00003036DD1403A41D351F8043B40F8043B6B
:1014B00051F8043B40F8043B51F8043B40F8043B2E
:1014C00051F8043B40F8043B51F8043B40F8043B1E
:1014D00051F8043B40F8043B51F8043B40F8043B0E
:1014E00051F8043B40F8043B51F8043B40F8043BFE
:1014F00051F8043B40F8043B51F8043B40F8043BEE
:1015000051F8043B40F8043B51F8043B40F8043BDD
:1015100051F8043B40F8043B51F8043B40F8043BCD
:1015200051F8043B40F8043B403ABDD2303211D36D
:1015300051F8043B40F8043B51F8043B40F8043BAD
:1015400051F8043B40F8043B51F8043B40F8043B9D
:10155000103AEDD20C3205D351F8043B40F8043B6D
:10156000043AF9D2043208D0D2071CBF11F8013B6B
:1015700000F8013B01D30B8803806046704700BF31
:10158000082A13D38B078DD010F003038AD0C3F140
:101590000403D21ADB071CBF11F8013B00F8013B22
:1015A00080D331F8023B20F8023B7BE7043AD9D3E1
:1015B000013A11F8013B00F8013BF9D20B780370B6
:1015C0004B7843708B788370604670474FEA410CCC
:1015D0007FEA6C5C02D150EA013C0AD14FEA430C2D
:1015E0007FEA6C5C02D152EA033C02D14FF000006A
:1015F00070474FF0010070474FEA410212F50012A8
:1016000015D211D56FF47873B3EB625212D94FEA49
:10161000C12343F0004343EA505311F0004F23FA33
:1016200002F018BF404270474FF00000704750EA88
:10163000013005D111F0004008BF6FF00040704745
:101640004FF00000704700BF70B58AB000230293CE
:101650000393022604960124059406930793094DEB
:1016600002A9284602F06CFC00942346324631461B
:10167000284602F0A7FC22462146284602F0BDFC7F
:101680000AB070BD7404002410B5FFF7DDFF054CEF
:10169000204602F0E1FC4FF470620349204602F05C
:1016A0007BFE10BD74040024020A801B2DE9F04764
:1016B00004460B46002942D1042A04D8DFE802F090
:1016C0003907272D33000026B146B24604E019261B
:1016D0004FF0AE094FF0020A0021A1600A251D2734
:1016E0004FF00108012B31D0204602F01BFDC4F859
:1016F00014A0C4F81C902662A661C4F82480E76296
:101700002563A562204602F0D1FABDE8F0871426D1
:101710004FF08B094FF0020ADEE714264FF08B09D9
:101720004FF0010AD8E714264FF03B094FF0010AA9
:10173000D2E714264FF08B094FF0040ACCE70025BE
:101740002F46A8462E46A946AA46CBE7053A042AC4
:1017500008D8DFE802F01F0310151A000625192724
:101760004FF001084FF44073A36014264FF03B097B
:101770004FF0010AB8E7052513274FF00108F1E7FC
:1017800005250E274FF00108ECE702250D274FF045
:101790000108E7E70A251D274FF00108E2E700B539
:1017A0008BB00191002102910391082B00D8049382
:1017B0000C2B1CD0102B1DD0142B1ED0182B1FD07F
:1017C000202B20D0302B21D0402B22D0002305937A
:1017D0004FF4801106914FF400110791089309937B
:1017E00001A902F0B4FCB8B90BB05DF804FB092103
:1017F0000491DFE70A210491DEE70B210491DDE784
:101800000C210491DCE70D210491DBE70E2104910A
:10181000DAE70F230493D9E70120E5E730B58BB071
:101820000C4613466A46402102F0CCFC18B1002554
:1018300028460BB030BD009B2380039B082B00D8AB
:10184000DDB2092B00D80C250A2B00D810250B2B54
:1018500000D814250C2B00D818250D2B00D82025D6
:101860000E2B00D830250F2BE2D84025E0E70000F2
:1018700008B5034B834200D008BD06F025FEFBE708
:101880007404002408B511F0007F04D00268936945
:1018900023F00103936111F4000F00D108BD00F0A3
:1018A0001FF8FFF7F1FEF9E700B583B00B4BD3F853
:1018B000D82042F00102C3F8D820D3F8D83003F082
:1018C00001030193019B002211460B2000F0C2FC92
:1018D0000B2000F0F1FC03B05DF804FB004402585B
:1018E00010B51648164B036000238360C360037471
:1018F0004374837401224261142181613B24C461D9
:1019000001624262022484620D22C2620463436364
:1019100004228263C2630A21016442648164C26456
:10192000046542658165C16501664366826602F0B1
:10193000BDF900B910BD00F0D3F8FBE77404002432
:1019400000A0004010B5B6B004460021319132919C
:10195000339134913591B82202A807F0FBFA22683E
:10196000294B9A4201D036B010BD4FF400420023FB
:10197000CDE902234FF080531D9302A803F056FFD8
:1019800000283ED1214BD3F8EC2042F48072C3F8FA
:10199000EC20D3F8EC2002F480720092009AD3F885
:1019A000E02042F00802C3F8E020D3F8E03003F072
:1019B00008030193019B03233193022332930024F4
:1019C000339434940923359331A9114802F0CCFEA5
:1019D00022462146132000F03DFC132000F06CFC51
:1019E00022462146152000F035FC152000F064FC4D
:1019F000224621463F2000F02DFC3F2000F05CFCF9
:101A0000B1E700F06DF8BDE700A0004000440258C7
:101A1000000C025808B502680C4B9A4200D008BD71
:101A20000B4AD2F8EC3023F48073C2F8EC30032177
:101A3000084802F089FF132000F04CFC152000F04C
:101A400049FC3F2000F046FCE9E700BF00A0004051
:101A500000440258000C025830B589B000240394A9
:101A600004940594069407941B4BD3F8E02042F0AD
:101A70008002C3F8E020D3F8E02002F08002009258
:101A8000009AD3F8E02042F00102C3F8E020D3F836
:101A9000E02002F001020192019AD3F8E02042F026
:101AA0000802C3F8E020D3F8E03003F00803029303
:101AB000029B0A4D22468021284602F0E9FF80233E
:101AC0000393012304930594069403A9284602F086
:101AD0004BFE09B030BD00BF004402580000025860
:101AE00072B6FEE700B59DB04C22002109A807F0B0
:101AF00031FA2022002101A807F02CFA022002F07E
:101B0000CDFF00230093204B9A6922F440429A6152
:101B10009B6903F440430093009B1B4B9B6913F4A8
:101B2000005FFAD0012209924FF480330A93022316
:101B3000129313931493282115911692062217924B
:101B400018930C23199300231A931B9309A802F0EE
:101B5000CFFFA8B93F2301930321029100230393F0
:101B6000082304934023059306934FF48062079261
:101B7000089301A803F0BEFB20B91DB05DF804FB7B
:101B8000FFF7AEFFFFF7ACFF0048025808B500F0C2
:101B9000FBFAFFF7A7FFFFF75FFFFFF785FEFFF7F1
:101BA0009FFE00F0F1F900F02BF900F063F907F067
:101BB00063F906F0B5FE3B4C042200212046FFF7F6
:101BC00075FDFFF761FD06F073F9374D2946204694
:101BD00006F056FD012000F017FB05F58871204640
:101BE00006F04EFD012000F00FFB05F508712046C0
:101BF00006F046FD012000F007FB05F54C7120467C
:101C000006F03EFD012000F0FFFA4FF47A7000F07C
:101C1000FBFA264804F0D4FD12E02146214806F0E4
:101C200033FE2FE022491F4806F02EFE2FE0214907
:101C30001C4806F029FE2FE01F491A4806F024FE32
:101C4000194C204606F0B8F9012000F0DDFA04F541
:101C5000887006F0B1F9012000F0D6FA04F508709A
:101C600006F0AAF9012000F0CFFA04F54C7006F056
:101C7000A3F9012000F0C8FA06F09CFE94F8583051
:101C8000002BCAD0084B93F86831002BCAD0064B02
:101C900093F87832002BCAD0034B93F88833002B8B
:101CA000CED1C9E774040024BC0600241405002426
:101CB000CC070024DC080024EC09002482B0074B88
:101CC000D3F8F42042F00202C3F8F420D3F8F43041
:101CD00003F002030193019B02B0704700440258D5
:101CE000FEE7FEE7FEE7FEE7FEE770477047704756
:101CF00008B500F077FA08BD08B5024801F00CFB02
:101D000008BD00BFAC05002408B5024802F09CFBEA
:101D100008BD00BF7404002408B5024802F094FB1B
:101D200008BD00BF7404002408B5024804F09CFDFF
:101D300008BD00BF1405002408B5024804F094FD56
:101D400008BD00BF6005002408B5024805F01CF975
:101D500008BD00BF2406002408B5024802F074FB49
:101D600008BD00BF740400241E4B1B6803F00F0362
:101D7000062B06D81B4A136823F00F0343F0070312
:101D80001360194B1A6842F001021A6000221A61AE
:101D90001968164A0A401A60124B1B6813F0080FA4
:101DA00006D0104A136823F00F0343F007031360B3
:101DB0000D4B00229A61DA611A620D4999620D4950
:101DC000D9620D4919635A639963DA6319645A64D5
:101DD000196821F4802119601A66084B43F2D20277
:101DE0001A60704700200052004402587FEDF6EA66
:101DF000000202020000FF018002010100400052C7
:101E000000B589B0002304930593069307930193CB
:101E1000029303931548164A0260EF2242608360E2
:101E200049F63F42C26003618023836104F070FE83
:101E300090B94FF48053049304A90C4804F0A4FE15
:101E400068B900230193039301A9084804F038FFFF
:101E500040B909B05DF804FBFFF742FEE9E7FFF780
:101E60003FFEEEE7FFF73CFEF3E700BF140500245A
:101E70000004004000B589B0002304930593069345
:101E800007930193029303931448154A0260EF22CB
:101E90004260836040F2E732C2600361836104F014
:101EA00037FE90B94FF48053049304A90B4804F013
:101EB0006BFE68B900230193039301A9074804F05E
:101EC000FFFE40B909B05DF804FBFFF709FEE9E742
:101ED000FFF706FEEEE7FFF703FEF3E760050024D9
:101EE0000008004000B583B003681A4A934205D049
:101EF000194A934218D003B05DF804FB174BD3F88E
:101F0000E82042F00202C3F8E820D3F8E83003F0FA
:101F100002030093009B002211461D2000F09AF955
:101F20001D2000F0C9F9E6E70C4BD3F8E82042F099
:101F30000402C3F8E820D3F8E83003F00403019367
:101F4000019B002211461E2000F084F91E2000F0A3
:101F5000B3F9D0E7000400400008004000440258F4
:101F600008B50268054B9A4200D008BD06F09AFFFA
:101F700027220349034804F043FFF6E7000400402A
:101F8000A41500242406002408B51748174B036045
:101F90004FF4E133436000238360C36003610C228C
:101FA00042618361C36103624362836205F049FE5B
:101FB00070B900210C4805F0BFFE60B900210A4845
:101FC00005F0DFFE50B9084805F097FE48B908BD96
:101FD000FFF786FDEDE7FFF783FDEFE7FFF780FDF5
:101FE000F1E7FFF77DFDF2E7240600240010014031
:101FF00030B5B7B00446002131913291339134911C
:102000003591B82202A806F0A5FF2268304B9A420B
:1020100001D037B030BD01220023CDE902230023D7
:10202000209302A803F002FC00284AD1294BD3F8E0
:10203000F02042F01002C3F8F020D3F8F02002F0B4
:1020400010020092009AD3F8E02042F00102C3F897
:10205000E020D3F8E03003F001030193019B4FF43B
:10206000C0633193022332930025339534950723BF
:10207000359331A9184802F077FB1848184B0360D4
:102080002A23436040238360C5604FF4806303616B
:1020900045618561C5610562042343620323836250
:1020A000C562056300F050FB70B90C4BE3679C639D
:1020B00000221146252000F0CDF8252000F0FCF884
:1020C000A7E7FFF70DFDB1E7FFF70AFDEDE700BF5A
:1020D000001001400044025800000258AC050024E2
:1020E00010000240DFF834D0FFF73EFE0C480D49E7
:1020F0000D4A002302E0D458C4500433C4188C4263
:10210000F9D30A4A0A4C002301E013600432A242C8
:10211000FBD306F0FBFEFFF739FD704700000524F6
:1021200000000024580400248CBB0008580400243C
:10213000F0150024FEE70000104B1B780BB90120BE
:10214000704710B504464FF47A70B0FBF3F30C4AB5
:102150001068B0FBF3F000F0CFF868B90F2C01D98C
:1021600001200AE0002221464FF0FF3000F072F813
:10217000044B1C60002000E0012010BD080000247A
:10218000000000240C00002410B5032000F050F8DB
:1021900002F0A4FF0F498B69C3F303230E4AD35CFB
:1021A00003F01F03D8408B6903F00F03D35C03F0E7
:1021B0001F0320FA03F3094A1360094B18600F202C
:1021C000FFF7BAFF10B10124204610BD0446FFF707
:1021D00075FDF9E700440258D4B500080400002456
:1021E00000000024034B1B78034A11680B44136062
:1021F000704700BF08000024B8060024014B18688F
:10220000704700BFB806002438B50446FFF7F6FF54
:102210000546B4F1FF3F02D0044B1B781C44FFF786
:10222000EDFF401BA042FAD338BD00BF08000024D8
:102230000649CB6823F4E0631B041B0C000200F486
:10224000E0600343024A1A43CA60704700ED00E0B1
:102250000000FA0530B4154BDB68C3F30223C3F169
:102260000704042C28BF04241D1D062D14D9033B8C
:102270004FF0FF3505FA04F421EA0401994005FA0C
:1022800003F322EA03031943002807DB0901C9B25B
:10229000074B195430BC70470023E9E700F00F00EA
:1022A0000901C9B2034B1954F4E700BF00ED00E087
:1022B00000E400E014ED00E0002807DB00F01F025E
:1022C000400901239340024A42F82030704700BF82
:1022D00000E100E000280CDB00F01F0240090123B0
:1022E00093402030034A42F82030BFF34F8FBFF3B2
:1022F0006F8F704700E100E00138B0F1807F0AD2B3
:10230000064B5860064AF02182F82310002098609E
:1023100007221A6070470120704700BF10E000E0FC
:1023200000ED00E0F0B4876D0468654E654DAC4289
:1023300018BFB44242D01835AC423FD01835AC4239
:102340003CD01835AC4239D01835AC4236D01835AF
:10235000AC4233D01835AC4230D005F55675AC429E
:102360002CD01835AC4229D01835AC4226D01835BF
:10237000AC4223D01835AC4220D01835AC421DD029
:102380001835AC421AD01835AC4217D04E4DAC427D
:1023900014D01435AC4211D01435AC420ED01435E3
:1023A000AC420BD01435AC4208D01435AC4205D049
:1023B0001435AC4202D01435AC4207D1446E856E60
:1023C0006560C46E14B1046F456F656004683C4E6F
:1023D0003C4DAC4218BFB44252D01835AC424FD03D
:1023E0001835AC424CD01835AC4249D01835AC4207
:1023F00046D01835AC4243D01835AC4240D005F534
:102400005675AC423CD01835AC4239D01835AC4288
:1024100036D01835AC4233D01835AC4230D01835F0
:10242000AC422DD01835AC422AD01835AC4227D05A
:10243000254E264DAC4218BFB44211D0244DAC42BB
:102440000ED01435AC420BD01435AC4208D0143544
:10245000AC4205D01435AC4202D01435AC4223D185
:10246000C46D04F01F050124AC407C600468636007
:102470008368402B1FD0036899600368DA6013E01B
:10248000C46D04F01F053F24AC40BC6005682C6897
:1024900024F480242C60046863608368402B05D09A
:1024A000036899600368DA60F0BC704703689A605B
:1024B0000368D960F8E703689A600368D960F3E7B6
:1024C0001000024028000240085402581C540258D0
:1024D0003054025803682749274A934218BF8B4259
:1024E0002FD0183293422CD01832934229D0183270
:1024F000934226D01832934223D01832934220D0F0
:10250000183293421DD002F55672934219D01832F8
:10251000934216D01832934213D01832934210D0FF
:10252000183293420DD0183293420AD01832934297
:1025300007D01832934204D023F0FF038365806DE7
:10254000704710B4D9B210390C4AA2FB0142C2F351
:1025500002120B4CA25CC2655F2906D9094A1A40D7
:1025600004328265806D10BC7047064A1A4082654D
:10257000F8E700BF1000024028000240ABAAAAAA58
:10258000E4B5000800FCFFFF83699BB9836A012B57
:102590000AD0022B02D00BB100207047C36A13F09F
:1025A000807F2AD100207047C36AB3F1C07F26D054
:1025B00000207047B3F5005F0AD0836A022B26D94A
:1025C000032B26D1C36A13F0807F24D100207047EB
:1025D000836A032B03D8DFE803F01404140A0020F5
:1025E0007047C36A13F0807F0DD100207047C36A23
:1025F000B3F1C07F09D0002070470120704701204F
:10260000704701207047012070470120704701206A
:10261000704700207047012070470000036822497E
:10262000224A934218BF8B4228D01432934225D0BD
:102630001432934222D0143293421FD01432934268
:102640001CD01432934219D01432934216D0DAB20D
:10265000103A1749A1FB0212120916491944A82978
:102660001FD9154B13449B000366144B436602F0BD
:102670001F02012303FA02F282667047DBB2083BB5
:102680000F4AA2FB03230F4A02EB131292000266C9
:102690000D4A4266C3F30413012202FA03F3836670
:1026A00070470832DDE700BF085402581C54025836
:1026B000ABAAAAAAF0FBFDBF00820010800802406E
:1026C000CDCCCCCC009600168058025801794A1E19
:1026D000072A2CD830B40368154D164CA34218BFF6
:1026E000AB4218D01434A34215D01434A34212D0F4
:1026F0001434A3420FD01434A3420CD01434A34298
:1027000009D01434A34206D00B4B0B449B00C36684
:102710000A4B036705E00A4B0B449B00C366094B59
:102720000367012303FA02F2426730BC7047704727
:10273000085402581C5402583F82001040090240BD
:102740003F9600164059025870B50446FFF756FDF3
:10275000002C00F0B58105462368AE49AE4A93428D
:1027600018BF8B420CBF0122002250D030318B4267
:102770004DD018318B424AD018318B4247D0183196
:102780008B4244D018318B4241D018318B423ED01D
:1027900001F556718B423AD018318B4237D018313F
:1027A0008B4234D018318B4231D018318B422ED02D
:1027B00018318B422BD018318B4228D018318B42E4
:1027C00025D09649964A934218BF8B4200F030813B
:1027D000944A934200F02C811432934200F02881F5
:1027E0001432934200F024811432934200F020818D
:1027F0001432934200F01C811432934200F018818D
:1028000040236365032384F8353001204AE0022128
:1028100084F83510002184F834107ABB824A934240
:102820002CD01832934229D01832934226D0183235
:10283000934223D01832934220D0183293421DD0B5
:1028400002F55672934219D01832934216D01832BC
:10285000934213D01832934210D0183293420DD0C5
:10286000183293420AD01832934207D0183293425A
:1028700004D01A6822F001021A6003E01A6822F0FC
:1028800001021A6023681A6812F0010F0BD0FFF7DB
:10289000B5FC431B052BF5D920236365032384F87E
:1028A0003530012070BD1A6860481040A168E268A8
:1028B0000A4321690A4361690A43A1690A43E1693C
:1028C0000A43216A0A430243616A042900F09680A0
:1028D0006168A1F12905A1F13F00032888BF052DFA
:1028E0000AD9A1F14700012806D9A1F14F00032818
:1028F00002D97439032901D842F480121A6026687B
:10290000756925F00705636A1D43042B08D1A36A86
:102910001D43E36A23B12046FFF736FE002872D13B
:1029200075612046FFF7D6FDE36D03F01F023F23DC
:102930009340836023683749374A934218BF8B42DC
:1029400042D0183293423FD0183293423CD01832D2
:10295000934239D01832934236D01832934233D052
:102960001832934230D002F5567293422CD018326E
:10297000934229D01832934226D01832934223D062
:102980001832934220D0183293421DD0183293420D
:102990001AD01832934217D0204A934214D01432DE
:1029A000934211D0143293420ED0143293420BD082
:1029B0001432934208D01432934205D01432934219
:1029C00002D01432934213D12046FFF727FEA368AA
:1029D000802B68D0236E22791A60636EA26E5A60D3
:1029E0006368013B072B61D90023E36623676367B4
:1029F00000206065012384F8353053E7E16A206BDD
:102A000001430A4364E740236365012084F83500ED
:102A100048E700BF10000240280002400854025856
:102A20001C54025830540258400002403F8010FEAF
:102A3000022284F83520002284F834201A682149C3
:102A40001140A268402A2CD0802A27D00022E068BA
:102A500042EAD002206942EAD002606942EAD0022A
:102A6000A06942EAD002E06942EAD002206A42EA62
:102A700010120A431A602268134B1344134AA2FB34
:102A800003231B099B00E3652046FFF723FDE26D4E
:102A900002F01F0101228A4042604BE74FF480425E
:102AA000D5E71022D3E70023636093E72046FFF7C2
:102AB0000DFEE36E00221A60236F626F5A6097E783
:102AC0000120EFE60F00FEFFF8ABFDA7CDCCCCCC8C
:102AD000002800F03E8170B5044690F834000128CB
:102AE00000F03981012084F8340094F83500C0B238
:102AF000012807D04FF400636365002384F8343065
:102B0000012070BD022084F8350000206065206837
:102B1000924E934DA84218BFB0422FD01835A8420C
:102B20002CD01835A84229D01835A84226D01835FF
:102B3000A84223D01835A84220D01835A8421DD06D
:102B400005F55675A84219D01835A84216D0183583
:102B5000A84213D01835A84210D01835A8420DD07D
:102B60001835A8420AD01835A84207D01835A8420F
:102B700004D0056825F00105056003E0056825F02F
:102B8000010505602046FFF7CDFB23687349744AB1
:102B9000934218BF8B4238D01832934235D0183246
:102BA000934232D0183293422FD0183293422CD015
:102BB0001832934229D01832934226D002F5567229
:102BC000934222D0183293421FD0183293421CD025
:102BD0001832934219D01832934216D018329342C9
:102BE00013D01832934210D0183293420DD01A6885
:102BF00022F00E0242F00A021A60236C93B122689E
:102C0000136843F0040313600CE01A6822F01E02FC
:102C100042F016021A60236C23B12268136843F055
:102C20000803136023684D494D4A934218BF8B42F5
:102C300042D0183293423FD0183293423CD01832DF
:102C4000934239D01832934236D01832934233D05F
:102C50001832934230D002F5567293422CD018327B
:102C6000934229D01832934226D01832934223D06F
:102C70001832934220D0183293421DD0183293421A
:102C80001AD01832934217D0364A934214D01432D5
:102C9000934211D0143293420ED0143293420BD08F
:102CA0001432934208D01432934205D01432934226
:102CB00002D0143293420ED1236E1A6812F4803F70
:102CC00003D01A6842F480721A60E36E1BB11A686E
:102CD00042F480721A6023682049214A934218BF47
:102CE0008B4230D0183293422DD0183293422AD0E2
:102CF0001832934227D01832934224D0183293428C
:102D000021D0183293421ED002F5567293421AD047
:102D10001832934217D01832934214D0183293428B
:102D200011D0183293420ED0183293420BD0183281
:102D3000934208D01832934205D01A6842F001023B
:102D40001A600020DDE61A6842F001021A600020D5
:102D5000D7E6012070470220D3E600BF10000240F2
:102D6000280002400854025870B50446FFF746FA9E
:102D7000002C00F09181054694F83530DBB2022B2F
:102D800006D080236365002384F83430012070BDB1
:102D900023688C498C4A934218BF8B4230D018323A
:102DA00093422DD0183293422AD01832934227D022
:102DB0001832934224D01832934221D018329342D1
:102DC0001ED002F5567293421AD01832934217D091
:102DD0001832934214D01832934211D018329342D1
:102DE0000ED0183293420BD01832934208D01832CA
:102DF000934205D01A6822F00E021A60266809E094
:102E00001A6822F01E021A602268536923F08003B8
:102E10005361266823686B496B4A934218BF8B4203
:102E200042D0183293423FD0183293423CD01832ED
:102E3000934239D01832934236D01832934233D06D
:102E40001832934230D002F5567293422CD0183289
:102E5000934229D01832934226D01832934223D07D
:102E60001832934220D0183293421DD01832934228
:102E70001AD01832934217D0544A934214D01432C5
:102E8000934211D0143293420ED0143293420BD09D
:102E90001432934208D01432934205D01432934234
:102EA00002D01432934204D1226E136823F480734B
:102EB000136023684349444A934218BF8B422FD082
:102EC000183293422CD01832934229D018329342B0
:102ED00026D01832934223D01832934220D0183291
:102EE00093421DD002F55672934219D01832934284
:102EF00016D01832934213D01832934210D01832A1
:102F000093420DD0183293420AD01832934207D020
:102F10001832934204D01A6822F001021A6003E0CA
:102F20001A6822F001021A60336813F0010F0ED004
:102F3000FFF764F9431B052BF6D9202363650323B0
:102F400084F83530002384F8343001201FE72368EB
:102F50001C491D4A934218BF8B4239D01832934204
:102F600036D01832934233D01832934230D01832D0
:102F700093422DD0183293422AD01832934227D050
:102F800002F55672934223D01832934220D0183261
:102F900093421DD0183293421AD01832934217D060
:102FA0001832934214D01832934211D018329342FF
:102FB0000ED0A16DE36D03F01F02012393404B601F
:102FC0000DE000BF100002402800024008540258E3
:102FD000A16DE36D03F01F023F2393408B602368D4
:102FE0002E492F4A934218BF8B4242D01832934247
:102FF0003FD0183293423CD01832934239D0183225
:10300000934236D01832934233D01832934230D0A4
:1030100002F5567293422CD01832934229D01832BE
:10302000934226D01832934223D01832934220D0B4
:10303000183293421DD0183293421AD0183293425C
:1030400017D0184A934214D01432934211D014323C
:1030500093420ED0143293420BD01432934208D0D4
:103060001432934205D01432934202D01432934268
:103070000BD1636EA26E5A60E36E33B11A6822F40C
:1030800080721A60236F626F5A60012384F83530B2
:10309000002084F834007AE6012078E6100002402F
:1030A0002800024008540258002800F0298108B581
:1030B000024690F83530DBB2022B03D08023436503
:1030C000012008BD0368904890498B4218BF834295
:1030D0000CBF0121002166D03030834263D018300C
:1030E000834260D0183083425DD0183083425AD07A
:1030F0001830834257D01830834254D000F55670B0
:10310000834250D0183083424DD0183083424AD089
:103110001830834247D01830834244D0183083425D
:1031200041D0183083423ED0183083423BD01968DA
:1031300021F00E0119601368A0F5956073498B4268
:1031400018BF83426AD072498B4267D018318B42D4
:1031500064D018318B4261D018318B425ED0183167
:103160008B425BD018318B4258D001F556718B429F
:1031700054D018318B4251D018318B424ED0183177
:103180008B424BD018318B4248D018318B4245D0FE
:1031900018318B4242D018318B423FD0196821F050
:1031A000010119603EE0042082F8350081BB584AD5
:1031B00093422DD0183293422AD01832934227D00E
:1031C0001832934224D01832934221D018329342BD
:1031D0001ED002F5567293421AD01832934217D07D
:1031E0001832934214D01832934211D018329342BD
:1031F0000ED0183293420BD01832934208D01832B6
:10320000934205D01A6822F001021A60002058E7A4
:103210001A6822F001021A60002052E7196821F0B2
:10322000010119601368384838498B4218BF83423E
:1032300042D018318B423FD018318B423CD01831EC
:103240008B4239D018318B4236D018318B4233D073
:1032500018318B4230D001F556718B422CD0183189
:103260008B4229D018318B4226D018318B4223D083
:1032700018318B4220D018318B421DD018318B422F
:103280001AD018318B4217D022498B4214D01431F6
:103290008B4211D014318B420ED014318B420BD0A3
:1032A00014318B4208D014318B4205D014318B423B
:1032B00002D014318B4217D1116E0B6823F4807346
:1032C0000B60906DD36D03F01F0101238B404360B1
:1032D000536E916E5960D36E33B1196821F48071C9
:1032E0001960136F516F5960012382F83530002344
:1032F00082F83430136D2BB1104698470020E0E679
:10330000012070470020DCE6100002402800024047
:103310004000024008540258F0B583B00446002330
:103320000193A24B1D68A24BA3FB0535AD0A876D27
:103330003E68D7F800C003689E499F48834218BF83
:103340008B420CBF0120002061D09C4A93425ED08A
:10335000183293425BD01832934258D018329342BD
:1033600055D01832934252D0183293424FD002F5C2
:10337000567293424BD01832934248D0183293423F
:1033800045D01832934242D0183293423FD018327F
:1033900093423CD01832934239D01832934236D0FF
:1033A0008749884A934218BF8B4212D0864A93427B
:1033B0000FD0143293420CD01432934209D01432FD
:1033C000934206D01432934203D01432934240F019
:1033D00062821A68E16D01F01F010420884010EA42
:1033E0000C0F00F0A88212F0040F00F0A4827860A5
:1033F00012F4004F00F05B8212F4803F40F05182E3
:10340000A36C002B00F047822046984743E2E26D10
:1034100002F01F0108228A40324241D070BB674A45
:1034200093422BD01832934228D01832934225D0A1
:103430001832934222D0183293421FD0183293424E
:103440001CD002F55672934218D01832934215D010
:103450001832934212D0183293420FD0183293424E
:103460000CD01832934209D01832934206D0183249
:10347000934203D01A68C2F3C00202E01A68C2F392
:1034800080026AB11A6822F004021A60E36D03F048
:103490001F0208239340BB60636D43F00103636523
:1034A000E26D02F01F0226FA02F313F0010F37D08B
:1034B0002368404840498B4218BF83422CD01831C2
:1034C0008B4229D018318B4226D018318B4223D021
:1034D00018318B4220D018318B421DD018318B42CD
:1034E0001AD001F556718B4216D018318B4213D089
:1034F00018318B4210D018318B420DD018318B42CD
:103500000AD018318B4207D018318B4204D01831C1
:103510008B4201D01B6803E05B6913F0800F3BD145
:10352000E36D03F01F03042202FA03F3334251D088
:103530002268204820498A4218BF824246D018316A
:103540008A4243D018318A4240D018318A423DD055
:1035500018318A423AD018318A4237D018318A421B
:1035600034D001F556718A4230D018318A422DD0BC
:1035700018318A422AD018318A4227D018318A421B
:1035800024D018318A4221D018318A421ED01831F5
:103590008A421BD013681DE0012303FA02F2BA60CD
:1035A000636D43F002036365BAE700BF00000024C7
:1035B000B5814E1B1000024028000240400002402E
:1035C000085402581C54025830540258126812F021
:1035D000020F3DD1E36D03F01F03102202FA03F343
:1035E00033425FD022689B489B498A4218BF82427F
:1035F00034D018318A4231D018318A422ED0183155
:103600008A422BD018318A4228D018318A4225D0DC
:1036100018318A4222D001F556718A421ED01831E3
:103620008A421BD018318A4218D018318A4215D0EC
:1036300018318A4212D018318A420FD018318A428A
:103640000CD018318A4209D01268C2F3800208E017
:10365000BB60636D43F004036365BBE71268C2F3AC
:10366000C002FAB1BB6023681A6812F4802F0DD033
:103670001B6813F4002F04D1236C9BB1204698479C
:1036800010E0A36C73B1204698470BE01A6812F45F
:10369000807F03D11A6822F008021A60236C0BB1F4
:1036A00020469847E36D03F01F03202202FA03F33C
:1036B000334200F08E802268664867498A4218BF0C
:1036C00082422ED018318A422BD018318A4228D01B
:1036D00018318A4225D018318A4222D018318A42C4
:1036E0001FD018318A421CD001F556718A4218D079
:1036F00018318A4215D018318A4212D018318A42C4
:103700000FD018318A420CD018318A4209D01831B2
:103710008A4206D018318A4203D01268C2F34002AE
:1037200002E01268C2F30012002A52D0BB6094F883
:103730003530DBB2042B0ED023681A6812F4802FC8
:1037400035D01B6813F4002F2CD1636C002B40D0B4
:10375000204698473DE02268136823F01603136063
:103760002268536923F080035361236CB3B122684C
:10377000136823F008031360E36D03F01F023F2377
:103780009340BB60012384F83530002384F8343043
:10379000236D002B7FD0204698477CE0A36C002B44
:1037A000E5D1E9E7E36BA3B12046984711E01A6839
:1037B00012F4807F09D11A6822F010021A600123E6
:1037C00084F83530002384F83430E36B0BB12046A5
:1037D0009847636D002B5ED0636D13F0010F56D0D8
:1037E000042384F8353023681A491B4A934218BFD2
:1037F0008B4233D01832934230D0183293422DD0BE
:10380000183293422AD01832934227D0183293426A
:1038100024D01832934221D002F5567293421DD023
:10382000183293421AD01832934217D0183293426A
:1038300014D01832934211D0183293420ED018325D
:1038400093420BD01832934208D01A6822F001023A
:103850001A6007E010000240280002401A6822F0B7
:1038600001021A60019B01330193AB4204D8236823
:103870001B6813F0010FF5D123681B6813F0010FCB
:103880000BD0032384F83530002384F83430E36C04
:103890000BB12046984703B0F0BD012384F83530C2
:1038A000F2E7236C002BF6D020469847F3E712F09E
:1038B000200F3AD123686449644A934218BF8B426F
:1038C0002FD0183293422CD01832934229D018327C
:1038D000934226D01832934223D01832934220D0FC
:1038E000183293421DD002F55672934219D0183205
:1038F000934216D01832934213D01832934210D00C
:10390000183293420DD0183293420AD018329342A3
:1039100007D01832934204D01A6822F004021A60C9
:1039200003E01A6822F008021A60236C002BB2D060
:1039300020469847AFE70220884010EA0C0F60D07D
:1039400012F0020F5DD0786012F4004F0ED012F426
:10395000803F05D1636C002B9DD0204698479AE7A5
:10396000E36B002B97D02046984794E712F0200F86
:1039700040D123683449354A934218BF8B422FD037
:10398000183293422CD01832934229D018329342E5
:1039900026D01832934223D01832934220D01832C6
:1039A00093421DD002F55672934219D018329342B9
:1039B00016D01832934213D01832934210D01832D6
:1039C00093420DD0183293420AD01832934207D056
:1039D0001832934204D01A6822F00A021A6003E0F7
:1039E0001A6822F014021A60012384F8353000238B
:1039F00084F83430E36B002B3FF44DAF20469847FA
:103A000049E7082000FA01F111EA0C0F3FF443AF37
:103A100012F0080F3FF43FAF1A6822F00E021A604E
:103A2000E36D03F01F03012202FA03F37B6062657A
:103A300084F83520002384F83430E36C002B3FF405
:103A40002AAF2046984726E710000240280002408F
:103A500030B4446B0268D2F88410704B194041EACC
:103A60008401C2F884100268D2F8841021F47F0126
:103A7000856B41EA0541C2F88410826B22440468D8
:103A8000D4F88810194041EA8201C4F8881004680B
:103A9000D4F8881021F4FE01C56B41EA0541C4F851
:103AA0008810C16B02EB41020468D4F8A0101940E1
:103AB00041EA8201C4F8A0100468D4F8A01021F4EF
:103AC000FE01056C41EA0541C4F8A010046C416C8C
:103AD00001FB04240268D2F8B010194041EA8401C5
:103AE000C2F8B0100268D2F8B01021F4FE01856C63
:103AF00041EA0541C2F8B010826CC16C01FB02447E
:103B00000268D2F8AC10194041EA8401C2F8AC1046
:103B1000026D416D01FB02420468D4F8F0101940B7
:103B200041EA8201C4F8F0100468D4F8F01021F4DE
:103B30007C11856D41EA0541C4F8F010816D02EBFE
:103B400041020468D4F8C0100B4043EA8202C4F872
:103B5000C0200268D2F8C03023F47C13C16D43EA60
:103B60000143C2F8C0300268D2F8C03023F07C5361
:103B7000016E43EA0163C2F8C030436B284A1A441D
:103B80009200C266836B02EB83030367C16B03EB96
:103B9000C1034367046C416C01FB04F103EB810337
:103BA0008367846CC16C01FB04F103EB8103C36781
:103BB000046D416D01FB04F103EB8103C0F880301B
:103BC000816D03EBC103C0F88430C46D856E05FBC5
:103BD00004F403EB8403C0F88830016E01FB05F1A7
:103BE00003EB8103C0F890300E498B4207D8D0F820
:103BF000903093420ED9002342F8043BF7E7D0F807
:103C00009C3043F02003C0F89C30032380F89830A8
:103C1000012000E0002030BC704700BF0300FFFF20
:103C2000002B0010FCD30040F0B44C68002C30D1C5
:103C30000E698C6826430C6846EA84460D6ACC6996
:103C400044EA05648D692C434D692C43CD6844EAF0
:103C50000544D0F88470806E03FB00F307EB830506
:103C600047F823606C6008350020CB680E4CE35C9D
:103C7000834216D91418E678A3781B0443EA066336
:103C8000647843EA0423145C234345F8043B04307E
:103C9000EBE70C698E6826430C68264346F08046A5
:103CA000CCE7F0BC704700BFECB5000830B595B06C
:103CB00004464C22A04901A8FDF7EEFB002C00F0C1
:103CC000388123689D4A934220D094F898300BB3F2
:103CD0002268936923F010039361FEF78FFA05467B
:103CE00023689A6912F0080F1AD0FEF787FA431B6F
:103CF0000A2BF5D9D4F89C3043F00103C4F89C306A
:103D0000032384F89830012015B030BD03F580738B
:103D10006360DAE784F899302046FDF713FED7E7B1
:103D20009A6942F001029A61FEF768FA0546236833
:103D30009A6912F0010F0FD1FEF760FA401B0A28B2
:103D4000F5D9D4F89C3043F00103C4F89C30032328
:103D500084F898300120D7E79A6942F002029A610C
:103D6000237C012B40D02268936943F04003936188
:103D7000637C012B3ED02268936923F480439361D6
:103D8000A37C012B3CD02268936943F48053936158
:103D90002268936923F44073A1680B4393612268FE
:103DA000936923F0A40393612268136923F010033D
:103DB0001361E368012B29D0002B2CD0022B00F0DB
:103DC0009B802268936943F08003936122681369A2
:103DD00043F010031361E368032B1CD1226893693D
:103DE00043F02003936116E02268936923F04003B7
:103DF0009361BDE72268936943F480439361BFE711
:103E00002268936923F480539361C1E72268936920
:103E100043F004039361A3695A1EE369013B1B024B
:103E200043EA4263226A013A13436269013A216814
:103E300043EA0243CB61A368B3F5407F62D0236EAF
:103E400033B12268D2F8C030616E0B43C2F8C03083
:103E5000E36D226ED3420DD02168D1F8C83023F033
:103E60000703A26E14A800EB820252F84C2C1343F5
:103E7000C1F8C830236C6BB12168D1F8BC3023F095
:103E80000703626C14A800EB820252F84C2C134317
:103E9000C1F8BC30A36C73B12168D1F8BC3023F0F9
:103EA0007003E26C14A800EB820252F84C2C43EA37
:103EB0000213C1F8BC30236D73B12168D1F8BC3056
:103EC00023F4E063626D14A800EB820252F84C2CDC
:103ED00043EA0223C1F8BC302268184B9A4222D030
:103EE0000023C4F89430C4F89C30012384F898303F
:103EF0002046FFF7ADFD07E72268936943F02003F2
:103F0000936188E7A36A013BE26A013A43EA02232C
:103F1000226B013A43EA0213626A013A216843EADA
:103F20000243CB608BE76268936823F003039360DE
:103F3000D6E70120E8E600BF88B5000800A00040F1
:103F400090F89830013BDBB2012B07D9D0F89C30B8
:103F500043F00203C0F89C3001207047CB680A6828
:103F6000D2B9072B0ED08A68DB0643EA82730A694E
:103F700043EA02434A691343C26E496842F821305A
:103F8000002070470A69CB691B0243EA02438A6931
:103F9000134343F06053EFE710B40A6942EA4372F7
:103FA000072B0DD08C684B6943EA8473006F496816
:103FB00000EBC10440F831206360002010BC704762
:103FC0008B69F3E710B490F89840E4B2012C08D064
:103FD000D0F89C3043F00403C0F89C30012010BCA2
:103FE0007047920042EA011242EA430203680199D3
:103FF0000A43C3F880200020F1E790F89830DBB244
:10400000012B07D0D0F89C3043F00403C0F89C305B
:104010000120704751B90168D1F8F03023F07C538A
:1040200043EA0262C1F8F02000207047012909D05C
:104030000168D1F8B03023F0FE4343EA0262C1F8D0
:10404000B020F1E70168D1F8A03023F0FE4343EA45
:104050000262C1F8A020E7E790F89830DBB2012BAC
:1040600007D0D0F89C3043F00403C0F89C30012006
:104070007047022380F898300268936923F00103A7
:1040800093610023C0F89C301846704790F8983030
:10409000DBB2022B3ED10268936943F001039361C6
:1040A00000230268916911F0010F0ED1322B01D863
:1040B0000133F6E7D0F89C3043F00103C0F89C30A0
:1040C000032380F8983001207047936923F0100390
:1040D000936100230268916911F0080F0ED0322B12
:1040E00001D80133F6E7D0F89C3043F00103C0F863
:1040F0009C30032380F8983001207047936943F087
:10410000020393610023C0F89430012280F89820C4
:1041100018467047D0F89C3043F00803C0F89C3034
:104120000120704788B110B50446FFF7AFFF226841
:10413000D36D23F00303D3652046FDF76BFC00200D
:10414000C4F89C0084F8980010BD0120704738B571
:10415000044690F89830DBB2022B2BD10368D3F8D9
:10416000C00010F07C5F0CD0D3F8C40010F4001F26
:104170000FD0D4F89C3043F40073C4F89C30012075
:104180001FE0D4F89C3043F02003C4F89C30012099
:1041900017E0D3F8C450C5F304452B462046FFF77B
:1041A00043FD22680123AB40C2F8D030C4F89430FC
:1041B000002006E0D0F89C3043F00803C0F89C30A3
:1041C000012038BDF0B490F89840E4B2022C40F0E1
:1041D000D88040290CD041293FD0046D8C4271D841
:1041E000D0F89C3043F02003C0F89C300120CFE091
:1041F0000468D4F8A05015F4FE0F0CD0D4F8A450E5
:1042000015F07F0F0FD1D0F89C3043F48073C0F8C5
:104210009C300120BCE0D0F89C3043F02003C0F873
:104220009C300120B4E0D4F8A450C5F3006C15F024
:10423000807F06D0D4F8A0505FEAD57C01D14FF042
:10424000000CD4F8A440C4F30524A444446F456C86
:104250000CFB05F504EB85043CE00468D4F8B05091
:1042600015F4FE0F0CD0D4F8B45015F07F0F0FD119
:10427000D0F89C3043F48073C0F89C30012087E074
:10428000D0F89C3043F02003C0F89C3001207FE040
:10429000D4F8B450C5F3006C15F0807F06D0D4F884
:1042A000B0505FEAD57C01D14FF0000CD4F8B44097
:1042B000C4F30524A444846FC56C0CFB05F504EB22
:1042C000850407E0C46F456D01FB05F504EB85042B
:1042D0004FF0000C256805F080455560002D2CD16D
:1042E0002568C5F38A451560256805F00055956079
:1042F000256805F000451561A588D561E58805F0BC
:104300000F05D560656805F480155561656805F48D
:1043100000159561E57905F07F0515626568ED0F7B
:10432000556204F108050024D6681A4FBE5DA64206
:1043300008D92E5D1E550134F6E7256825F0604545
:104340001560D1E740290AD041290DD01F290FD887
:104350000268012303FA01F1C2F8981002E0036831
:10436000C3F8A8C0002013E00368C3F8B8C0F9E799
:1043700001F01F010268012303FA01F1C2F89C1049
:10438000F0E7D0F89C3043F00803C0F89C300120DF
:10439000F0BC7047ECB5000890F89830013BDBB2F8
:1043A000012B07D9D0F89C3043F00203C0F89C30B1
:1043B0000120704710B403689C6D0C4223D1DC6D62
:1043C00044F00104DC6511F4007F05D00468D4F8E2
:1043D000E0301343C4F8E03011F4806F05D0046876
:1043E000D4F8E4301A43C4F8E4200068436D0C4A62
:1043F0000A40134343650B4A536943EA9171516183
:10440000002010BC70479C6D31EA040402D00324E4
:10441000DC65D8E7DC6D44F00204DC65D3E700BF5F
:10442000FFFFCF3F00A800407047704770477047BC
:1044300070477047704770477047704770477047C4
:1044400070477047704700002DE9F04F83B0044675
:10445000B74B1A695B699B0703EA82730193036890
:104460001A6D02F4704A5A6D0AEA020A1A6D02F0D5
:104470000F095A6D09EA02091A6D02F0F0085A6D27
:1044800008EA02081E6D06F071565A6D16401F6D3F
:1044900007F060775A6D17405D6DD3F850B015F492
:1044A000807F02D01BF4807F64D115F4806F02D02E
:1044B0001BF4806F67D1019B002B74D1BAF1000F00
:1044C0007CD1B9F1000F40F08580B8F1000F40F0C9
:1044D0008D8015F4006F03D01BF4006F40F09280C4
:1044E00015F4007F03D01BF4007F40F0968015F494
:1044F000002F03D01BF4002F40F09F8015F4803F65
:1045000003D01BF4803F40F0A38015F4802F03D02C
:104510001BF4802F40F0A78015F4003F0FD01BF450
:10452000003F0CD023684FF400321A65804B002204
:104530001A61D4F89C3043F08003C4F89C30002FFB
:1045400040F09C804EB123681E65B20F784B1A6113
:10455000D4F89C301E43C4F89C602268754B9A4284
:1045600000F09680D4F89C30002B40F0F88003B027
:10457000BDE8F08F4FF480721A656D4B00221A610E
:10458000FFF75BFF91E72368D3F8DC10D3F8E42052
:104590004FF480601865664B00201861114020467A
:1045A000FFF747FF87E7236800221A6501998A0F02
:1045B0005F4B1A612046FFF737FF7FE72368C3F898
:1045C00050A04FEA9A725A4B1A6151462046FFF7A3
:1045D0002CFF76E72368C3F850904FEA9972544B4A
:1045E0001A6149462046FDF743F96EE72368C3F890
:1045F00050804FEA98724E4B1A6141462046FFF7B1
:1046000015FF66E723684FF400621A65484B0022E5
:104610001A612046FFF70BFF62E72368D3F8D81032
:10462000D3F8E0204FF400701865414B002018616A
:1046300011402046FFF7FCFE59E723684FF40022A3
:104640001A653B4B00221A612046FFF7F3FE55E73F
:1046500023684FF480321A65354B00221A612046D8
:10466000FFF7E9FE51E723684FF480221A65304BCB
:1046700000221A612046FFF7DFFE4DE723681F6521
:10468000BA0F2B4B1A6139462046FDF7FBF859E764
:1046900063689A6812F0030F3FF464AF196A01F07F
:1046A0000F015A6A186A00F03008586A08EA0008D0
:1046B0001F6A07F4C077586A07401E6A06F4FC4672
:1046C000586A06401D6A05F4F025586A0540D3F87B
:1046D0002490D3F820A011401CD1B8F1000F1ED1B6
:1046E00019F0400F02D01AF0400F25D187BB36B128
:1046F00063681E62D4F89C301E43C4F89C60002D91
:104700003FF430AF63681D62D4F89C301D43C4F899
:104710009C5027E719622046FFF791FEDDE76368AA
:10472000C3F8208041462046FFF78AFED8E700BF45
:1047300000A8004000A000406368D96BDA6B4020FD
:10474000186202F03F02090C2046FFF77AFECDE71F
:1047500063681F6239462046FFF774FEC7E72046AC
:10476000FFF76CFE03E700BFF0B482B000235FE008
:1047700086685F000325BD4026EA0506CD68BD407A
:1047800035438560466826EA04064D68C5F3001483
:104790009C403443446059E0DD08083550F82570EA
:1047A00003F00704A6000F24B44027EA04070C69AD
:1047B000B4403C4340F825405CE0092400E000247C
:1047C000B4403C4302355C4E46F825404FF0B044BF
:1047D0002568D44325EA02064F6817F4801F01D0EC
:1047E00042EA05064FF0B0452E606E6804EA060501
:1047F0004F6817F4001F01D042EA06054FF0B0469B
:1048000075604E4D6D6804EA05064F6817F4003F69
:1048100001D042EA0506494D6E602D682C404E6875
:1048200016F4803F01D042EA0504444A1460013383
:104830000A6832FA03F47BD001249C402240F6D06F
:104840004D6805F00305013D012D91D94C6804F038
:104850000304032C09D0C5685E000324B44025EA94
:1048600004058C68B4402C43C4604C6804F0030415
:10487000022C91D005685E000324B44025EA0405AB
:104880004C6804F00304B4402C4304604C6814F4F6
:10489000403FCCD02A4CD4F8F45045F00205C4F87F
:1048A000F450D4F8F44004F002040194019C9D08F3
:1048B000AE1C214C54F8267003F00304A6000F240C
:1048C000B44027EA04071F4CA0423FF478AF04F538
:1048D0008064A0421ED004F58064A0421CD004F580
:1048E0008064A0421AD004F58064A04218D004F578
:1048F0008064A04216D004F58064A04214D004F570
:104900008064A04212D004F50064A0423FF455AF89
:104910000A2455E7012453E7022451E703244FE713
:1049200004244DE705244BE7062449E7072447E71D
:1049300002B0F0BC704700BF00040058800000586F
:104940000044025800000258002390E0092600E0CD
:10495000002606FA04F4AC426BD005685C0003261E
:1049600006FA04F42543056023FA06F5083550F8E5
:10497000256003F007074FEA870C0F2707FA0CF7AB
:1049800026EA070640F82560C56825EA0405C560E3
:10499000456825EA02024260826822EA04048460D3
:1049A000013331FA03F260D001229A4012EA010C7D
:1049B000F6D09F08BD1C334C54F8255003F0030477
:1049C000A4000F2606FA04FE0EEA05052E4EB0429C
:1049D000BED006F58066B0421DD006F58066B042B6
:1049E0001BD006F58066B04219D006F58066B0424D
:1049F00017D006F58066B04215D006F58066B04245
:104A000013D006F58066B04211D006F50066B042BC
:104A10009CD00A269DE701269BE7022699E70326FC
:104A200097E7042695E7052693E7062691E70726EC
:104A30008FE7164C256825EA0C052560656825EA90
:104A40000C0565604FF0B044656825EA0C056560AB
:104A5000256825EA0C0525600A4DBC1C55F8246024
:104A600026EA0E0645F8246077E7F0BD013331FAF7
:104A700003F206D001229A4012EA010CF6D0F0B5FA
:104A800097E7704700040058000002588000005863
:104A90000AB181617047090481617047134BDB687B
:104AA00013F0040F07D1114BDB6803F007038342B7
:104AB0001AD00120704710B50C4AD36823F00703C1
:104AC0001843D060FDF79AFB0446084B5B6813F46B
:104AD000005F07D1FDF792FB001BB0F57A7FF4D998
:104AE000012000E0002010BD00207047004802585F
:104AF000002800F0D78238B50446036813F0010F90
:104B000025D0AA4A136903F03803926A102B15D0F6
:104B1000182B0FD06368B3F5803F3FD0002B53D1E3
:104B2000A24B1A6822F480321A601A6822F480229A
:104B30001A6038E002F00302022AEBD19B4B1B689B
:104B400013F4003F03D06368002B00F0AD822368AC
:104B500013F0020F00F08880944A1369926A13F0F0
:104B600038035AD0182B55D0E368002B00F0A980E9
:104B70008E490A6822F0190213430B60FDF73EFBD1
:104B800005468A4B1B6813F0040F40F09180FDF737
:104B900035FB401B0228F4D903208CE2834A1368BA
:104BA00043F48033136063682BB3FDF727FB05469E
:104BB0007E4B1B6813F4003FC9D1FDF71FFB401B60
:104BC0006428F5D9032076E2B3F5A02F09D0774BFE
:104BD0001A6822F480321A601A6822F480221A605D
:104BE000E1E7724B1A6842F480221A601A6842F4B4
:104BF00080321A60D7E7FDF701FB05466B4B1B6857
:104C000013F4003FA3D0FDF7F9FA401B6428F5D94F
:104C1000032050E212F0030FA6D1644B1B6813F07F
:104C2000040F03D0E368002B00F040825F4A136852
:104C300023F01903E1680B431360FDF7DFFA054623
:104C40005A4B1B6813F0040F06D1FDF7D7FA401B2F
:104C50000228F5D903202EE2544A536823F0FE437C
:104C6000216943EA01635360236813F0100F51D0A8
:104C70004E4A136903F03803926A082B39D0182B77
:104C800033D0E369002B68D0484A136843F08003AF
:104C90001360FDF7B3FA0546444B1B6813F4807F9D
:104CA00052D1FDF7ABFA401B0228F5D9032002E2EE
:104CB0003E4A536823F0FE43216943EA016353608F
:104CC000D2E73A4A136823F001031360FDF796FA1E
:104CD0000546364B1B6813F0040FC5D0FDF78EFA5E
:104CE000401B0228F5D90320E5E102F00302012A66
:104CF000C7D12E4B1B6813F4807F03D0E369802B50
:104D000040F0D681294AD36823F07C53216A43EAD4
:104D10000163D360236813F0080F49D0636983B33C
:104D2000224A536F43F001035367FDF767FA0546C4
:104D30001E4B5B6F13F0020F3AD1FDF75FFA401B79
:104D40000228F5D90320B6E1184AD36823F07C5332
:104D5000216A43EA0163D360DCE7144A136823F055
:104D600080031360FDF74AFA0546104B1B6813F4E5
:104D7000807FCFD0FDF742FA401B0228F5D90320EF
:104D800099E10A4A536F23F001035367FDF736FA9E
:104D90000546064B5B6F13F0020F09D0FDF72EFAA4
:104DA000401B0228F5D9032085E100BF00440258CA
:104DB000236813F0200F29D0A3699BB1A84A136878
:104DC00043F480531360FDF719FA0546A44B1B68A2
:104DD00013F4005F1AD1FDF711FA401B0228F5D930
:104DE000032068E19E4A136823F480531360FDF7A3
:104DF00005FA05469A4B1B6813F4005F06D0FDF7D1
:104E0000FDF9401B0228F5D9032054E1236813F073
:104E1000040F21D1636A002B00F04C81904A126983
:104E200002F03802182A00F0EA80022B75D08C4A72
:104E3000136823F080731360FDF7E0F90446884B94
:104E40001B6813F0007F00F0D880FDF7D7F9001B36
:104E50000228F4D903202EE1824A136843F48073B8
:104E60001360FDF7CBF905467E4B1B6813F4807F7A
:104E700006D1FDF7C3F9401B6428F5D903201AE1D8
:104E8000A368012B0AD00BBB754B1A6F22F00102ED
:104E90001A671A6F22F004021A6704E0704A136F4F
:104EA00043F001031367A36833B3FDF7A7F9054681
:104EB0006B4B1B6F13F0020FACD1FDF79FF9401B3A
:104EC00041F288339842F3D90320F4E0052B09D04E
:104ED000634B1A6F22F001021A671A6F22F0040264
:104EE0001A67E0E75E4B1A6F42F004021A671A6F06
:104EF00042F001021A67D6E7FDF780F90546584BE4
:104F00001B6F13F0020F85D0FDF778F9401B41F2BB
:104F100088339842F3D90320CDE0514A136823F037
:104F200080731360FDF76AF905464D4B1B6813F05B
:104F3000007F06D0FDF762F9401B0228F5D9032057
:104F4000B9E0474B996A484A0A40A16AE06A41EAD7
:104F500000110A439A62226B013AC2F30802616BA4
:104F60000139490289B20A43A16B0139090401F4EC
:104F7000FE010A43E16B0139090601F0FE410A43D3
:104F80001A63DA6A22F00102DA62596B374A0A4080
:104F9000A16C42EAC1025A63DA6A22F00C02216C67
:104FA0000A43DA62DA6A22F00202616C0A43DA62C8
:104FB000DA6A42F48032DA62DA6A42F40032DA62A1
:104FC000DA6A42F48022DA62DA6A42F00102DA62D4
:104FD0001A6842F080721A60FDF710F90446204BFF
:104FE0001B6813F0007F06D1FDF708F9001B0228AB
:104FF000F5D903205FE000205DE000205BE0184968
:105000008A6A086B012B57D002F00303A16A8B4216
:1050100054D1C2F30512E36A9A4251D1C0F3080297
:10502000236B013B9A424DD1C0F34622636B013B97
:105030009A4249D1C0F30642A36B013B9A4245D143
:10504000C0F30660E36B013B984241D1044B5B6BBC
:10505000C3F3CC03A26C9A420AD100202BE000BF1C
:1050600000440258004802580CFCFFFF0700FFFFF5
:10507000184AD36A23F00103D362FDF7BFF805464F
:10508000FDF7BCF8A842FBD0124A516B124B0B4003
:10509000A16C43EAC1035363D36A43F00103D362B3
:1050A000002008E001207047012004E0012002E018
:1050B000012000E0002038BD0120FCE70120FAE7D4
:1050C0000120F8E70120F6E70120F4E70120F2E7EC
:1050D0000120F0E7004402580700FFFFF8B57E4BBF
:1050E0001B6903F03803102B00F0F280182B10D04E
:1050F00013B17A4C2046F8BD774B1B6813F0200F94
:1051000000F0E880744B1868C0F3C100744CC440D0
:10511000F0E7714B9D6A05F003059C6AC4F3051422
:10512000D86A00F001005B6BC3F3CC0300FB03F013
:10513000FBF74AFE0646002CDCD0012D76D0022D6E
:1051400000F0A4800DB32046FBF73EFE0146654803
:10515000FBF746FF0446604B186BC0F30800FBF7F3
:1051600033FE05464FF064513046FBF785FE01469D
:105170002846FBF779FD4FF07E51FBF775FD0146A0
:105180002046FBF779FE044671E0534B1B6813F091
:10519000200F29D0504F3B68C3F3C1035048D8407B
:1051A000FBF712FE05462046FBF70EFE0146284699
:1051B000FBF716FF0446386BC0F30800FBF704FE4C
:1051C00005464FF064513046FBF756FE014628462F
:1051D000FBF74AFD4FF07E51FBF746FD01462046A6
:1051E000FBF74AFE044642E02046FBF7EDFD014690
:1051F0003D48FBF7F5FE0446374B186BC0F308003B
:10520000FBF7E2FD05464FF064513046FBF734FEF4
:1052100001462846FBF728FD4FF07E51FBF724FDA1
:1052200001462046FBF728FE044620E02046FBF717
:10523000CBFD01462B48FBF7D3FE0446264B186BEB
:10524000C0F30800FBF7C0FD05464FF0645130463F
:10525000FBF712FE01462846FBF706FD4FF07E5194
:10526000FBF702FD01462046FBF706FE04461A4BFB
:105270001B6BC3F34623581CFBF7A6FD01462046D3
:10528000FBF7AEFEFBF76EFF044633E72046FBF765
:105290009BFD01461548FBF7A3FE04460E4B186B19
:1052A000C0F30800FBF790FD05464FF0645130460F
:1052B000FBF7E2FD01462846FBF7D6FC4FF07E5196
:1052C000FBF7D2FC01462046FBF7D6FD0446CEE7AD
:1052D000074C0FE7024C0DE70044025800093D005F
:1052E0000090D0030024744A0024744C001BB74B78
:1052F00000366E01002800F0328170B50D4604467C
:105300009B4B1B6803F00F038B420BD2984A136828
:1053100023F00F030B431360136803F00F038B425A
:1053200040F01F81236813F0040F0CD02269914BC9
:105330009B6903F070039A4205D98E498B6923F06B
:1053400070031A438A61236813F0080F0CD0626956
:10535000884BDB6903F070039A4205D98549CB6914
:1053600023F070031A43CA61236813F0100F0CD0A6
:10537000A269804BDB6903F4E0639A4205D97D4959
:10538000CB6923F4E0631A43CA61236813F0200F4A
:105390000CD0E269774B1B6A03F070039A4205D97F
:1053A00074490B6A23F070031A430A62236813F0EE
:1053B000020F0CD0E2686F4B9B6903F00F039A4217
:1053C00005D96C498B6923F00F031A438A6123685E
:1053D00013F0010F41D0674A936923F47063A16809
:1053E0000B4393616368022B0AD0032B27D0012B58
:1053F0002CD0604A126812F0040F06D10120ADE0F3
:10540000126812F4003F00F0AE805A490A6922F097
:10541000070213430B61FCF7F1FE0646554B1B696F
:1054200003F038036268B3EBC20F16D0FCF7E6FE58
:10543000801B41F288339842F0D903208EE04D4A18
:10544000126812F0007FE0D1012087E0494A12681B
:1054500012F4807FD9D1012080E0236813F0020F7D
:105460000CD0E268434B9B6903F00F039A4205D2CC
:1054700040498B6923F00F031A438A613C4B1B6838
:1054800003F00F03AB420AD9394A136823F00F0324
:105490002B431360136803F00F03AB4265D12368FD
:1054A00013F0040F0CD02269324B9B6903F0700398
:1054B0009A4205D22F498B6923F070031A438A61FF
:1054C000236813F0080F0CD062692A4BDB6903F0E4
:1054D00070039A4205D22749CB6923F070031A431F
:1054E000CA61236813F0100F0CD0A269214BDB694D
:1054F00003F4E0639A4205D21E49CB6923F4E063CA
:105500001A43CA61236813F0200F0CD0E269194BCB
:105510001B6A03F070039A4205D216490B6A23F006
:1055200070031A430A62FFF7D9FD12498B69C3F36E
:105530000323114AD35C03F01F03D8408B6903F0A7
:105540000F03D35C03F01F0320FA03F30B4A13602D
:105550000B4B18600B4B1868FCF7EEFD70BD01207B
:1055600070470120FAE70120F8E70120F6E700BFC5
:105570000020005200440258D4B500080400002462
:10558000000000240C00002408B5FFF7A7FD0B4A1B
:105590009369C3F303230A49CB5C03F01F0320FA8A
:1055A00003F3926902F00F02885C00F01F0023FAF7
:1055B00000F0044A1060044A136008BD0044025819
:1055C000D4B50008040000240000002408B5FFF74B
:1055D000DBFF054BDB69C3F30213044AD35C03F022
:1055E0001F03D84008BD00BF00440258D4B50008CE
:1055F00008B5FFF7C9FF054BDB69C3F30223044A73
:10560000D35C03F01F03D84008BD00BF004402581C
:10561000D4B50008404B9B6A03F00303032B79D0F9
:1056200070B505460E463C4A136823F0806313604C
:10563000FCF7E4FD0446384B1B6813F0006F06D0FE
:10564000FCF7DCFD031B022BF5D9032070BD324BA8
:105650009A6A22F47C32296842EA01329A626A68C4
:10566000013AC2F30802A9680139490289B20A4322
:10567000E9680139090401F4FE010A432969013985
:10568000090601F0FE410A439A63DA6A22F0C00279
:1056900069690A43DA62DA6A22F02002A9690A43D8
:1056A000DA62DA6A22F01002DA62D96B1B4A0A4027
:1056B000E96942EAC102DA63DA6A42F01002DA62A8
:1056C000C6B91A46DB6A43F40023D362124A136850
:1056D00043F080631360FCF791FD04460E4B1B689A
:1056E00013F0006F14D1FCF789FD001B0228F5D9D7
:1056F0000320ABE7012E05D0074AD36A43F4001319
:10570000D362E3E7044AD36A43F48013D362DDE74C
:1057100000209BE701207047004402580700FFFF6C
:10572000404B9B6A03F00303032B79D070B5054609
:105730000E463C4A136823F080531360FCF75EFD6D
:105740000446384B1B6813F0005F06D0FCF756FD8B
:10575000031B022BF5D9032070BD324B9A6A22F04D
:105760007C72296842EA01529A626A68013AC2F37D
:105770000802A9680139490289B20A43E968013976
:10578000090401F4FE010A4329690139090601F0FF
:10579000FE410A431A64DA6A22F4406269690A43E4
:1057A000DA62DA6A22F40072A9690A43DA62DA6A12
:1057B00022F48072DA62596C1B4A0A40E96942EAB3
:1057C000C1025A64DA6A42F48072DA62C6B91A46D1
:1057D000DB6A43F48003D362124A136843F08053B8
:1057E0001360FCF70BFD04460E4B1B6813F0005FC3
:1057F00014D1FCF703FD001B0228F5D90320ABE709
:10580000012E05D0074AD36A43F08073D362E3E7E1
:10581000044AD36A43F40003D362DDE700209BE728
:1058200001207047004402580700FFFFF8B5044606
:10583000016801F000620023134330D0436EB3F5DA
:10584000001F26D00ED8EBB1B3F5801F07D102217F
:105850000830FFF7DFFE054645B12E4621E0012660
:1058600035461EE0B3F5401F09D10025A84A136D47
:1058700023F44013616E0B431365002611E00126EB
:1058800035460EE0A24AD36A43F40033D3620025C2
:10589000ECE702212830FFF743FF0546DCE700264E
:1058A0003546216801F480720023134314D0A36DA0
:1058B000042B37D8DFE803F003282F080800944AA8
:1058C000D36A43F40033D3627DBB914A136D23F056
:1058D0000703A16D0B431365216801F48062002367
:1058E000134336D0D4F8A430B3F5800F55D021D867
:1058F000002B4CD0B3F5001F19D1002104F1080092
:10590000FFF788FE05461BE0002104F10800FFF7C1
:1059100081FE0546D8E7002104F12800FFF700FFCB
:105920000546D1E701263546D6E72E46D4E70126BF
:1059300035460EE0B3F5000F02D0B3F5200F20D1AD
:1059400095BB734A936D23F46003D4F8A4100B4302
:105950009365216801F400620023134339D0D4F821
:10596000A830B3F1007F5CD023D8002B53D0B3F123
:10597000807F1BD1002104F10800FFF74BFE054694
:105980001DE0B3F5C00FDBD001263546E1E7604AE4
:10599000D36A43F40033D362D2E7002104F1280034
:1059A000FFF7BEFE0546CBE72E46D2E70126354679
:1059B0000FE0B3F1806F02D0B3F1A06F25D1002DBD
:1059C00036D1534A936D23F0E063D4F8A8100B430B
:1059D0009365216801F000720023134331D0E36C1A
:1059E000202B45D029D833B1102B23D1484AD36A74
:1059F00043F40033D362002D41D1454AD36C23F0E8
:105A00003003E16C0B43D3641BE0B3F1407FD6D08D
:105A100001263546DDE73E4AD36A43F40033D362BC
:105A2000CDE7002104F12800FFF77AFE0546C6E71E
:105A30002E46CEE70126354603E0302BDBD001268B
:105A40003546216801F48052002313432BD0E36DC7
:105A5000B3F5005F4FD017D8002B46D0B3F5805F69
:105A60000FD1002104F10800FFF7D4FD054611E035
:105A7000022104F10800FFF7CDFD0546BBE72E46E5
:105A8000DFE7012635460EE0B3F5405F02D0B3F5FF
:105A9000804F27D1002D35D11D4A136D23F4E043EB
:105AA000E16D0B431365216801F400520023134399
:105AB0003BD0236EB3F5003F58D02BD843B1B3F59C
:105AC000803F21D1012104F10800FFF7A3FD054625
:105AD000002D52D10E4A136D23F4E023216E0B43A7
:105AE000136522E001263546DDE7094AD36A43F40F
:105AF0000033D362CEE7002104F12800FFF710FE47
:105B00000546C7E72E46CEE7012635460DE000BF25
:105B100000440258B3F5802FDAD0B3F5A02FD7D0C8
:105B2000B3F5403FD4D001263546216801F48042C8
:105B30000023134331D0D4F8AC30B3F1005F49D027
:105B400020D843B1B3F1805F19D1012104F10800DD
:105B5000FFF760FD0546002D43D1954A936D23F074
:105B6000E043D4F8AC100B43936516E0012104F137
:105B70002800FFF7D5FD0546AAE72E46D5E7012602
:105B800035460AE0B3F1804FE5D0B3F1A04FE2D043
:105B9000B3F1405FDFD001263546216801F40042B1
:105BA0000023134309D0E36EB3F1805F1BD0B3F140
:105BB000005F26D0E3B101263546216801F08072EE
:105BC000002313433FD0A36C032B38D8DFE803F046
:105BD00027223027012104F12800FFF7A1FD054607
:105BE000B9E72E46D9E7724AD36A43F40033D36249
:105BF00075B96F4A136D23F04053E16E0B43136583
:105C0000DBE7012104F10800FFF704FD0546EFE79B
:105C10002E46D2E7664AD36A43F40033D3628DB985
:105C2000634AD36C23F00303A16C0B43D3640AE0F3
:105C3000022104F10800FFF7EDFC0546EFE701261D
:105C4000354600E02E46216801F48002002313430C
:105C500021D1216801F001020023134300F0978055
:105C6000A36F282B00F29180DFE803F07F8F8F8FE6
:105C70008F8F8F8F798F8F8F8F8F8F8F888F8F8F51
:105C80008F8F8F8F7F8F8F8F8F8F8F8F7F8F8F8F44
:105C90008F8F8F8F7F00474A136843F480731360A0
:105CA000FCF7ACFA0746434B1B6813F4807F05D121
:105CB000FCF7A4FAC01B6428F5D90325002D4AD1AE
:105CC0003B4B1B6FD4F8B020534013F4407F0CD0F3
:105CD000374B1A6F22F44072196F41F48031196703
:105CE000196F21F4803119671A67D4F8B030B3F511
:105CF000807F15D08DBBD4F8B03003F44072B2F57C
:105D0000407F1ED02A4A136923F47C53136128492B
:105D10000B6FD4F8B020C2F30B0213430B6798E764
:105D2000FCF76CFA0746224B1B6F13F0020FE1D110
:105D3000FCF764FAC01B41F288339842F3D903257B
:105D4000D8E71B48026922F47C521B4901EA13136D
:105D500013430361DBE72E467BE72E4679E70121FB
:105D600004F10800FFF756FC0546F5B9104A536DDB
:105D700023F03803A16F0B43536508E0012104F1C0
:105D80002800FFF7CDFC0546EFE7012635462168E0
:105D900001F00202002313432AD0636F052B23D89E
:105DA000DFE803F0120C1B1212122E46EFE700BFC1
:105DB0000044025800480258CFFFFF00012104F1BF
:105DC0000800FFF727FC05468DB9B54A536D23F04F
:105DD0000703616F0B4353650AE0012104F12800BA
:105DE000FFF79EFC0546EFE70126354600E02E460C
:105DF000216801F004020023134323D0D4F890302B
:105E0000052B1BD8DFE803F0090313090909012159
:105E100004F10800FFF7FEFB054695B9A04A936D13
:105E200023F00703D4F890100B4393650AE0012197
:105E300004F12800FFF774FC0546EEE7012635461D
:105E400000E02E46216801F020020023134328D0F1
:105E5000D4F88C30B3F1005F44D017D843B1B3F11C
:105E6000805F10D1002104F10800FFF7D3FB054645
:105E7000002D3ED18A4A536D23F0E043D4F88C10B4
:105E80000B4353650DE0012635460AE0B3F1804F20
:105E9000EED0B3F1A04FEBD0B3F1405FE8D00126D4
:105EA0003546216801F040020023134331D0D4F875
:105EB0009830B3F5006F4FD020D843B1B3F5806F61
:105EC00019D1002104F10800FFF7A4FB0546002DBD
:105ED00049D1734A936D23F4E053D4F898100B43DF
:105EE000936516E0022104F12800FFF719FC05462E
:105EF000BEE72E46D5E7012635460AE0B3F5805FBA
:105F0000E5D0B3F5A05FE2D0B3F5406FDFD0012656
:105F10003546216801F080020023134333D0D4F8C2
:105F20009C30B3F5804F00F0B28021D843B1B3F577
:105F3000005F1AD1002104F10800FFF76BFB054652
:105F4000002D40F0AB80564A936D23F46043D4F8A3
:105F50009C100B43936516E0022104F12800FFF723
:105F6000DFFB0546B3E72E46D3E7012635460AE0B8
:105F7000B3F5004FE4D0B3F5204FE1D0B3F5C04FF7
:105F8000DED001263546216801F0080200231343C4
:105F90000DD0D4F88030B3F5805F00F08380404AA4
:105FA000536D23F44053D4F880100B43536521689C
:105FB00001F01002002313430CD0D4F89430B3F551
:105FC000807F79D0364A936D23F44073D4F89410CF
:105FD0000B439365216801F40022002313430CD086
:105FE000D4F8A030B3F5803F00F08080B3F5003FD7
:105FF00072D0002B6AD001263546216801F4802238
:10600000002313430DD0D4F88430B3F5001F00F003
:106010008580B3F5401F77D0B3F5801F6FD0012680
:106020003546216801F480320023134308D0236DE4
:10603000002B7CD0B3F5803F00F0878001263546E9
:10604000216801F000520023134340F0878021684B
:1060500001F400320023134300F08D80E36FB3F5A9
:10606000807F00F0F78040F28380B3F5007F03D09B
:10607000B3F5407F40F0EC80002D40F0F180084AFD
:10608000536D23F44073E16F0B43536573E00221BA
:1060900004F12800FFF744FB054651E72E4672E75E
:1060A00000440258022104F12800FFF739FB0028C0
:1060B0003FF475AF012672E7022104F12800FFF7D3
:1060C0002FFB00283FF47EAF01267BE7002104F17F
:1060D0000800FFF79FFA05467DB97D4A936D23F4CA
:1060E0004033D4F8A0100B43936586E7022104F1F6
:1060F0002800FFF715FB0546EEE72E467DE7744ABC
:10610000D36A43F40033D3627DB9714A536D23F4EB
:106110004013D4F884100B43536582E7012104F146
:106120002800FFF7FDFA0546EEE72E4679E7684AB4
:10613000D36A43F40033D36275B9654AD36C23F450
:106140008033216D0B43D3647AE7022104F1080008
:10615000FFF760FA0546EFE72E4671E7022104F1EA
:106160002800FFF7DDFA00283FF471AF01266EE743
:10617000002B81D00126216801F4801200231343F3
:1061800006D0534A136D23F00043216F0B43136570
:10619000216801F400120023134306D04C4A136D0A
:1061A00023F08073A16E0B431365216801F08042D8
:1061B0000023134309D0464B1A6922F400421A61A6
:1061C0001A69D4F8B4100A431A61216801F0004238
:1061D0000023134306D03E4AD36C23F04053616D35
:1061E0000B43D364216801F400020023134307D05A
:1061F000374A536D23F44003D4F888100B4353659A
:106200006168002201F0010313432BD16168002271
:1062100001F0020313432ED16168002201F0040350
:10622000134331D16168002201F00803134334D1D4
:106230006168002201F01003134337D16168002226
:1062400001F0200313433AD106B101263046F8BDD0
:10625000012690E71E4AD36A43F40033D3620BE76A
:106260002E4688E7002104F10800FFF7D3F9002843
:10627000CCD00646CAE7012104F10800FFF7CAF9AD
:106280000028C9D00646C7E7022104F10800FFF73D
:10629000C1F90028C6D00646C4E7002104F1280051
:1062A000FFF73EFA0028C3D00646C1E7012104F1FA
:1062B0002800FFF735FA0028C0D00646BEE70221C5
:1062C00004F12800FFF72CFA0028BDD00646BBE7F2
:1062D0000044025808B5FFF757F9054B1B6AC3F392
:1062E0000213044AD35C03F01F03D84008BD00BF6B
:1062F00000440258D4B500082DE9F0410446864B0D
:106300009D6A9E6AC6F30536D86AC0F30010DB6B3F
:10631000C3F3CC0300FB03F0FAF756FD002E00F0A8
:10632000F58005F003050746012D79D0022D00F018
:10633000CB800DB33046FAF747FD01467748FAF7B0
:106340004FFE0546744B986BC0F30800FAF73CFD0E
:1063500006464FF064513846FAF78EFD0146304646
:10636000FAF782FC4FF07E51FAF77EFC0146284690
:10637000FAF782FD054674E0674B1B6813F0200FA7
:106380002CD0DFF89481D8F80030C3F3C1036448FF
:10639000D840FAF719FD05463046FAF715FD0146D3
:1063A0002846FAF71DFE0546D8F83800C0F3080065
:1063B000FAF70AFD06464FF064513846FAF75CFDDD
:1063C00001463046FAF750FC4FF07E51FAF74CFC8C
:1063D00001462846FAF750FD054642E03046FAF7F6
:1063E000F3FC01464F48FAF7FBFD05464A4B986B14
:1063F000C0F30800FAF7E8FC06464FF0645138464F
:10640000FAF73AFD01463046FAF72EFC4FF07E517E
:10641000FAF72AFC01462846FAF72EFD054620E049
:106420003046FAF7D1FC01463C48FAF7D9FD05465B
:10643000394B986BC0F30800FAF7C6FC06464FF0DC
:1064400064513846FAF718FD01463046FAF70CFC5D
:106450004FF07E51FAF708FC01462846FAF70CFD8A
:1064600005462D4EB06BC0F34620FAF7ADFC4FF059
:106470007E51FAF7F9FB01462846FAF7B1FDFAF723
:1064800071FE2060B06BC0F30640FAF79DFC4FF040
:106490007E51FAF7E9FB01462846FAF7A1FDFAF723
:1064A00061FE6060B06BC0F30660FAF78DFC4FF0E0
:1064B0007E51FAF7D9FB01462846FAF791FDFAF723
:1064C00051FEA060BDE8F0813046FAF77DFC014640
:1064D0001548FAF785FD05460F4B986BC0F3080089
:1064E000FAF772FC06464FF064513846FAF7C4FCDE
:1064F00001463046FAF7B8FB4FF07E51FAF7B4FB8D
:1065000001462846FAF7B8FC0546AAE700232360AF
:106510006360A360D6E700BF004402580024744AB9
:106520000090D0030024744C001BB74B2DE9F041C0
:106530000446864B9D6A9E6AC6F30556D86AC0F328
:1065400000205B6CC3F3CC0300FB03F0FAF73CFCC8
:10655000002E00F0F58005F003050746012D79D0E7
:10656000022D00F0CB800DB33046FAF72DFC01462A
:106570007748FAF735FD0546744B186CC0F30800F0
:10658000FAF722FC06464FF064513846FAF774FCDD
:1065900001463046FAF768FB4FF07E51FAF764FB8C
:1065A00001462846FAF768FC054674E0674B1B680D
:1065B00013F0200F2CD0DFF89481D8F80030C3F30B
:1065C000C1036448D840FAF7FFFB05463046FAF7A6
:1065D000FBFB01462846FAF703FD0546D8F84000C4
:1065E000C0F30800FAF7F0FB06464FF06451384656
:1065F000FAF742FC01463046FAF736FB4FF07E517F
:10660000FAF732FB01462846FAF736FC054642E027
:106610003046FAF7D9FB01464F48FAF7E1FC054648
:106620004A4B186CC0F30800FAF7CEFB06464FF051
:1066300064513846FAF720FC01463046FAF714FB5D
:106640004FF07E51FAF710FB01462846FAF714FC8A
:10665000054620E03046FAF7B7FB01463C48FAF71A
:10666000BFFC0546394B186CC0F30800FAF7ACFBC9
:1066700006464FF064513846FAF7FEFB01463046B5
:10668000FAF7F2FA4FF07E51FAF7EEFA0146284691
:10669000FAF7F2FB05462D4E306CC0F34620FAF7B0
:1066A00093FB4FF07E51FAF7DFFA01462846FAF7DE
:1066B00097FCFAF757FD2060306CC0F30640FAF7FC
:1066C00083FB4FF07E51FAF7CFFA01462846FAF7DE
:1066D00087FCFAF747FD6060306CC0F30660FAF79C
:1066E00073FB4FF07E51FAF7BFFA01462846FAF7DE
:1066F00077FCFAF737FDA060BDE8F0813046FAF785
:1067000063FB01461548FAF76BFC05460F4B186C06
:10671000C0F30800FAF758FB06464FF064513846BC
:10672000FAF7AAFB01463046FAF79EFA4FF07E517F
:10673000FAF79AFA01462846FAF79EFB0546AAE7B9
:10674000002323606360A360D6E700BF00440258C3
:106750000024744A0090D0030024744C001BB74BF3
:1067600030B4036A056A25F001050562846924F0E6
:10677000F00444EA021423F00A030B438461036229
:1067800030BC704730B4036A056A25F01005056215
:10679000846924F4704444EA023423F0A00343EAF9
:1067A00001138461036230BC704700008268034BB0
:1067B00013400B4343F00703836070478FFFCFFF05
:1067C00090F83D30DBB2012B42D1022380F83D30FE
:1067D0000268D36843F00103D36003681E4AB3F133
:1067E000804F18BF934225D0A2F57C42934221D01E
:1067F00002F5806293421DD002F58062934219D067
:1068000002F57842934215D0A2F56C42934211D022
:1068100002F5943293420DD0A2F5C042934209D0C2
:1068200002F58062934205D01A6842F001021A60B4
:10683000002070479968094A0A40062A18BFB2F535
:10684000803F07D01A6842F001021A6000207047AA
:106850000120704700207047000001400700010040
:10686000704770477047704770B504460368DE682C
:106870001D6915F0020F10D016F0020F0DD06FF049
:1068800002021A610123037703689B6913F0030F67
:1068900064D0FFF7E6FF0023237715F0040F12D032
:1068A00016F0040F0FD023686FF004021A61022360
:1068B000237723689B6913F4407F55D02046FFF768
:1068C000D0FF0023237715F0080F12D016F0080F21
:1068D0000FD023686FF008021A610423237723681E
:1068E000DB6913F0030F46D02046FFF7BAFF002301
:1068F000237715F0100F12D016F0100F0FD0236869
:106900006FF010021A61082323772368DB6913F400
:10691000407F37D02046FFF7A4FF0023237715F0F0
:10692000010F02D016F0010F33D115F4025F02D02F
:1069300016F0800F35D115F4807F02D016F0800F4D
:1069400037D115F0400F02D016F0400F39D115F0B5
:10695000200F02D016F0200F3BD170BDFFF780FF53
:106960002046FFF77FFF96E72046FFF779FF204696
:10697000FFF778FFA5E72046FFF772FF2046FFF7F5
:1069800071FFB4E72046FFF76BFF2046FFF76AFF71
:10699000C3E723686FF001021A612046FBF7E0FAB3
:1069A000C3E723686FF402521A61204600F0E1F950
:1069B000C1E723686FF480721A61204600F0DAF9AB
:1069C000BFE723686FF040021A612046FFF74BFFD4
:1069D000BDE723686FF020021A61204600F0C8F975
:1069E000BBE7000070B40368404CA04214BF002411
:1069F0000124B0F1804F14BF224644F00102AAB92D
:106A00003B4DA84214BF002501253A4EB0420DD09F
:106A100065B905F1804505F58235A84214BF00250A
:106A2000012506F50066B04200D01DB123F07003C9
:106A30004D682B4362BB2E4A904214BF00220122B4
:106A40002C4DA84224D01ABB02F1804202F58232BA
:106A5000904214BF0022012205F50065A84217D01C
:106A6000B2B9254A904214BF0022012205F59A3599
:106A7000A8420DD062B9214A904214BF00220122DF
:106A800005F50065A84203D012B91D4A904203D112
:106A900023F44073CA68134323F080034A69134305
:106AA00003608A68C2620A688262164B984214BF09
:106AB000234644F001035BB90F4B984214BF0023F7
:106AC0000123114A904203D013B9104B984201D1CF
:106AD0000B69036301234361036913F0010F03D0C2
:106AE000036923F00103036170BC7047000001409B
:106AF00000080040000400400044014000E0004065
:106B000000E4004000040140004001400048014012
:106B100060B310B5044690F83D3013B3022384F8F7
:106B20003D30214651F8040BFFF75CFF012384F848
:106B3000483084F83E3084F83F3084F8403084F8A0
:106B4000413084F8423084F8433084F8443084F88B
:106B5000453084F8463084F8473084F83D300020D2
:106B600010BD80F83C30FBF7BDF9D7E70120704736
:106B700010B4846824F47F4442EA03220A43224387
:106B8000826010BC7047000090F83C30012B00F090
:106B90008F8010B50446012380F83C30022380F832
:106BA0003D3002689068434B034093600B68702B44
:106BB00055D031D8502B6CD00CD9602B2AD1CA6853
:106BC00049682068FFF7DEFD60212068FFF7EEFDD1
:106BD000002035E0402B0AD1CA6849682068FFF7D9
:106BE000BFFD40212068FFF7E1FD002028E05BD8D1
:106BF000202B07D003D9302B04D0012020E00BB18B
:106C0000102B05D119462068FFF7D0FD002017E0B2
:106C1000012015E0012013E0B3F5005F2CD00BD963
:106C2000254A9342EED012D9244A9342EAD0103238
:106C30009342E7D0012003E0B3F5805F36D1002016
:106C4000012384F83D30002384F83C3010BDB3F5B7
:106C5000801FD7D0B3F1101FD4D00120F0E7CB684C
:106C60004A6889682068FFF783FF2268936843F0C9
:106C7000770393600020E3E7CB684A68896820685F
:106C8000FFF776FF2268936843F480439360002007
:106C9000D6E7CA6849682068FFF762FD502120687E
:106CA000FFF784FD0020CBE70120C9E70120C7E7FB
:106CB000022070478800CEFF200010003000100036
:106CC00090F83C30012B4DD070B4012380F83C305B
:106CD000022380F83D3003685A689D68224E234C99
:106CE000A34218BFB34203D122F470024C6822437E
:106CF00022F070020C6822435A6003681A4AB3F10A
:106D0000804F18BF93421FD0A2F57C4293421BD004
:106D100002F58062934217D002F58062934213D04D
:106D200002F5784293420FD0A2F56C4293420BD009
:106D300002F59432934207D0A2F5C042934203D0A9
:106D400002F58062934204D125F080058A681543DC
:106D50009D60012380F83D30002380F83C301846C8
:106D600070BC7047022070470000014000040140E1
:106D7000704770477047026852E8003F23F0C00335
:106D800042E800310029F6D1026802F1080353E815
:106D9000003F23F40003083242E800310029F3D118
:106DA0002023C0F888307047026852E8003F23F47F
:106DB000907342E800310029F6D1026802F108031D
:106DC00053E8001F0D4B0B40083242E80031002908
:106DD000F3D1C36E012B06D02023C0F88C300023E2
:106DE000C36643677047026852E8003F23F0100310
:106DF00042E800310029F6D1EEE700BFFEFFFFEFC9
:106E00001346D0F88820202A40D110B50446B3FAA2
:106E100083F25209002908BF0122002A38D10165F6
:106E2000A0F85430A0F85630C0F890202122C0F8C5
:106E30008820C26FCAB11749D163C26F1649116465
:106E4000C26F1649D164C26F0021116502682832F1
:106E5000016DC06FFBF73CFE38B11023C4F89030D1
:106E60002023C4F8883001200FE0236840221A62F2
:106E7000226802F1080353E8003F43F08003083220
:106E800042E800310029F3D1002010BD02207047F4
:106E90000120FAE7A36E00080F6F00081B6F0008BF
:106EA000704708B50346806BDB69B3F5807F18D067
:106EB0000023A0F85630026802F1080353E8003FAF
:106EC00023F08003083242E800310029F3D1026840
:106ED00052E8003F43F0400342E800310029F6D178
:106EE00008BDFFF7DDFFFBE708B5026852E8003F89
:106EF00023F0400342E800310029F6D12023C0F8F6
:106F0000883000238367FFF7CBFF08BD704708B5C3
:106F1000806BFFF7FBFF08BD704738B5846BD4F872
:106F20008820D4F88C5023689B6813F0800F01D020
:106F3000212A10D023689B6813F0400F01D0222D26
:106F400010D0D4F8903043F01003C4F890302046AD
:106F5000FFF7E2FF38BD0023A4F856302046FFF7C4
:106F60000AFFE7E70023A4F85E302046FFF71CFF86
:106F7000E7E708B5806B0023A0F85E30A0F8563034
:106F8000FFF7CAFF08BD704770B504460168CB69BA
:106F900008688D6840F60F021A4008D113F0200FE0
:106FA00005D010F0200F34D115F0805F31D12AB117
:106FB000B34A2A4033D1B34E304230D1E26E012A77
:106FC00000F0C68013F4801F03D015F4800F40F04A
:106FD0009B8113F0800F07D010F0800F40F09B8151
:106FE00015F4000F40F0978113F0400F03D010F01C
:106FF000400F40F0978113F4000F03D010F0804F42
:1070000040F0948113F0807F02D00028C0F292817A
:1070100070BD636F002BFBD020469847F8E713F054
:10702000010F09D010F4807F06D001260E62D4F83B
:1070300090103143C4F8901013F0020F0BD015F0EC
:10704000010F08D0216802260E62D4F8901041F09A
:107050000401C4F8901013F0040F0BD015F0010FC9
:1070600008D0216804260E62D4F8901041F0020185
:10707000C4F8901013F0080F0BD010F0200F00D1BF
:107080003AB1226808211162D4F890200A43C4F86A
:10709000902013F4006F0CD010F0806F09D022689C
:1070A0004FF400611162D4F8902042F02002C4F83D
:1070B0009020D4F89020002AAAD013F0200F09D0F5
:1070C00010F0200F02D115F0805F03D0636F0BB179
:1070D00020469847D4F8902023689B6813F0400F0F
:1070E00002D112F0280F2CD02046FFF75DFE236856
:1070F0009B6813F0400F20D0226802F1080353E888
:10710000003F23F04003083242E800310029F3D168
:10711000D4F880306BB15C4A1A65D4F88000FBF774
:10712000C3FF00283FF474AFD4F88000036D984784
:107130006EE72046FFF7F0FE6AE72046FFF7ECFE19
:1071400066E72046FFF7E8FE0023C4F890305FE7CB
:1071500013F0100F3FF436AF10F0100F3FF432AFC2
:1071600010230B6223689B6813F0400F00F092809D
:10717000D4F880201368454845498B4218BF8342A4
:107180002DD018318B422AD018318B4227D018319C
:107190008B4224D018318B4221D018318B421ED023
:1071A00018318B421BD001F556718B4217D0183124
:1071B0008B4214D018318B4211D018318B420ED033
:1071C00018318B420BD018318B4208D018318B42CA
:1071D00005D018318B4202D05B689BB201E05B683E
:1071E0009BB2002B3FF414AFB4F85C1099427FF6C9
:1071F0000FAFA4F85E30D369B3F5807F32D0226838
:1072000052E8003F23F4807342E800310029F6D1B0
:10721000226802F1080353E8003F23F0010308321B
:1072200042E800310029F3D1226802F1080353E853
:10723000003F23F04003083242E800310029F3D137
:107240002023C4F88C300023E366226852E8003F14
:1072500023F0100342E800310029F6D1D4F8800071
:10726000FBF782FD02232367B4F85C10B4F85E30AC
:107270009BB2C91A89B22046FFF785FEC8E600BF57
:107280000100001020010004736F0008100002408C
:1072900028000240B4F85C10B4F85E309BB2C91A02
:1072A00089B2B4F85E309BB2002B3FF4B1AE002936
:1072B0003FF4AEAE226852E8003F23F4907342E8F8
:1072C00000300028F6D1226802F1080353E8000FCD
:1072D0001A4B0340083242E800300028F3D1202343
:1072E000C4F88C300023E3666367226852E8003FED
:1072F00023F0100342E800300028F6D10223236770
:107300002046FFF740FE83E64FF480130B622046D1
:1073100000F0F0FC7CE6A36F002B3FF479AE204632
:10732000984775E62046FFF7DFFD71E6204600F03E
:10733000E3FC6DE6204600F0DEFC69E6FEFFFFEFB1
:107340002DE9F04186B00446016883680269134361
:1073500042691343C26913430868914A02401343C8
:107360000B602268536823F44053E1680B43536079
:10737000A16922688B4B9A4201D0236A1943906815
:10738000894B03400B4393602268D36A23F00F03B9
:10739000616A0B43D3622268844B9A4229D0844BA2
:1073A0009A4200F09480834B9A4200F0AA80824B6C
:1073B0009A4200F0C080814B9A4200F0D680804B08
:1073C0009A4200F009817F4B9A4200F02E817E4B59
:1073D0009A4200F041817D4B9A4200F054817C4BEF
:1073E0009A4200F079816F4B9A4200F09E8180238F
:1073F00033E0784B5B6D03F03803282B65D8DFE86A
:1074000013F02900640064006400640064006400F8
:107410006400AC0164006400640064006400640003
:1074200064002B0064006400640064006400640075
:1074300064005E0064006400640064006400640032
:107440006400600064006400640064006400640020
:1074500064006200012300E0082352498A4200F0E0
:107460009581E069B0F5004F00F00D82202B00F20D
:107470006682202B00F2BA82DFE813F087028D02C9
:10748000B802B8029002B802B802B8029502B80277
:10749000B802B802B802B802B802B8029A02B8023A
:1074A000B802B802B802B802B802B802B802B8020C
:1074B000B802B802B802B802B802B802A602102395
:1074C000CBE72023C9E74023C7E78023C5E7414B2B
:1074D0005B6D03F00703052B11D8DFE813F00600FE
:1074E000400108000A000C000E000023B5E7082345
:1074F000B3E71023B1E72023AFE74023ADE78023B4
:10750000ABE7344B5B6D03F00703052B11D8DFE8C5
:1075100013F00600280108000A000C000E000023EA
:107520009BE7082399E7102397E7202395E740235B
:1075300093E7802391E7274B5B6D03F00703052B4F
:1075400011D8DFE813F00600100108000A000C0053
:107550000E00002381E708237FE710237DE7202327
:107560007BE7402379E7802377E71A4B5B6D03F0D5
:107570000703052B11D8DFE813F00600F800080018
:107580000A000C000E00002367E7082365E71023BC
:1075900063E7202361E740235FE780235DE700BFC7
:1075A000F369FFCF000C0058FFF4FF1100100140F9
:1075B0000044004000480040004C004000500040A3
:1075C0000014014000780040007C00400018014099
:1075D000001C014000440258694B5B6D03F0380306
:1075E000282B20D8DFE803F0151F1F1F1F1F1F1FA8
:1075F000C31F1F1F1F1F1F1F171F1F1F1F1F1F1FFF
:10760000191F1F1F1F1F1F1F1B1F1F1F1F1F1F1F94
:107610001D00012321E708231FE710231DE7202376
:107620001BE7402319E7802317E7554B5B6D03F0F9
:107630000703052B0ED8DFE803F0039C0507090BB1
:1076400000230AE7082308E7102306E7202304E7BE
:10765000402302E7802300E7494B5B6D03F00703FB
:10766000052B0ED8DFE803F003870507090B00237D
:10767000F3E60823F1E61023EFE62023EDE64023AE
:10768000EBE68023E9E63E4B5B6D03F03803282BE5
:1076900020D8DFE803F0151F1F1F1F1F1F1F721FB9
:1076A0001F1F1F1F1F1F171F1F1F1F1F1F1F191FF8
:1076B0001F1F1F1F1F1F1B1F1F1F1F1F1F1F1D00FF
:1076C0000123CAE60823C8E61023C6E62023C4E641
:1076D0004023C2E68023C0E6294B5B6D03F03803EC
:1076E000282B20D8DFE803F0151F1F1F1F1F1F1FA7
:1076F0004E1F1F1F1F1F1F1F171F1F1F1F1F1F1F73
:10770000191F1F1F1F1F1F1F1B1F1F1F1F1F1F1F93
:107710001D000123A1E608239FE610239DE62023F8
:107720009BE6402399E6802397E603F50E339B6D95
:1077300003F00703052B0ED8DFE803F00326050747
:10774000090B022389E6082387E6102385E6202318
:1077500083E6402381E680237FE604237DE604233D
:107760007BE6042379E6042377E6042375E6042305
:1077700073E6042371E604236FE604236DE600BF7D
:1077800000440258042368E6042366E6202B27D829
:10779000022BC0F01D81023B1E2B00F21B81DFE893
:1077A00013F05200190158001901190119015D0067
:1077B00019011901190119011901190119016200B1
:1077C00019011901190119011901190119011901E9
:1077D00019011901190119011901190119016E0085
:1077E000402B2ED14FF40040626A824B33F81220B6
:1077F000B0FBF2F3656805EB4501994200F2EC80BD
:10780000B3EB053F00F2EA804FF0000892B200238C
:107810004146F9F7C7FC0F0247EA106706026808FD
:107820002A464346301847F10001F9F7BBFCA0F5A2
:107830004072714B9A4200F2D3802368D860404670
:1078400098E0012096E0FEF745FD0028CCD100200D
:1078500090E003A8FEF750FD0498F6E76846FEF7AF
:1078600065FE0198F1E7654B1B6813F0200F08D007
:10787000624B1B68C3F3C1036148D840E5E7614828
:10788000B2E75F48B0E7202B15D8202B00F2AA8082
:10789000DFE803F03238A8A83BA8A8A840A8A8A809
:1078A000A8A8A8A845A8A8A8A8A8A8A8A8A8A8A8BB
:1078B000A8A8A8A85100402B1CD1626A4D4B33F8F0
:1078C0001230B0FBF3F06268530803EB4000B0FBEA
:1078D000F2F0A0F110024FF6EF739A4200F28480AA
:1078E00083B223F00F03C0F3420018432368D8602B
:1078F00000203FE001203DE0FDF768FE0028DCD1DC
:10790000002037E0FDF774FEF8E703A8FEF7F4FC6B
:107910000498F3E76846FEF709FE0198EEE7374B57
:107920001B6813F0200F08D0344B1B68C3F3C1034E
:107930003348D840E2E73348BFE73148BDE7402B42
:1079400017D14FF40040626A2A4B33F81230B0FB73
:10795000F3F0636800EB5300B0FBF3F0A0F110020A
:107960004FF6EF739A4243D8236880B2D860002064
:1079700000E001200123A4F86A30A4F86830002355
:107980006367A36706B0BDE8F081FDF71FFE00281E
:10799000D9D10020EEE7FDF72BFEF8E703A8FEF7AC
:1079A000ABFC0498F3E76846FEF7C0FD0198EEE7EC
:1079B000124B1B6813F0200F08D0104B1B68C3F349
:1079C000C1030F48D840E2E70E48BCE70C48BAE7CD
:1079D0000120CFE70120CDE70120CBE70120C9E757
:1079E0000120C7E70120C5E70120C3E70120C1E767
:1079F0000120BFE7FCB50008FFFC0F00004402585F
:107A00000090D00300093D00836A13F0080F06D0F0
:107A10000268536823F40043816B0B435360836A0D
:107A200013F0010F06D00268536823F40033C16AD3
:107A30000B435360836A13F0020F06D00268536849
:107A400023F48033016B0B435360836A13F0040FFC
:107A500006D00268536823F48023416B0B435360C4
:107A6000836A13F0100F06D00268936823F48053E2
:107A7000C16B0B439360836A13F0200F06D002683A
:107A8000936823F40053016C0B439360836A13F0F3
:107A9000400F0AD00268536823F48013416C0B43F3
:107AA0005360436CB3F5801F0BD0836A13F0800FD3
:107AB00006D00268536823F40023C16C0B43536063
:107AC00070470268536823F4C003816C0B43536012
:107AD000EBE72DE9F84305460E4617469946DDF8D3
:107AE00020802C68E46936EA04030CBF01240024DA
:107AF000BC423AD1B8F1FF3FF3D0FAF77FFBA0EBDD
:107B00000900404534D8B8F1000F33D02B681A680B
:107B100012F0040FE5D0B6F1400218BF0122802E0A
:107B2000DFD0002ADDD0DA6912F0080F11D1DA694E
:107B300012F4006FD5D04FF400621A622846FFF7A6
:107B400033F92023C5F89030002385F884300320D2
:107B50000CE008241C622846FFF726F9C5F890407F
:107B6000002385F88430012000E00020BDE8F88380
:107B70000320FBE70320F9E730B583B00446002378
:107B8000C0F89030FAF73AFB054623681B6813F0FB
:107B9000080F10D123681B6813F0040F28D120238D
:107BA000C4F88830C4F88C300020E066206784F880
:107BB000840003B030BD6FF07E4300930346002283
:107BC0004FF400112046FFF784FF0028E2D022681E
:107BD00052E8003F23F0800342E800310029F6D14B
:107BE0002023C4F88830002384F884300320E0E7A1
:107BF0006FF07E4300932B4600224FF48001204615
:107C0000FFF767FF0028CAD0226852E8003F23F43C
:107C1000907342E800310029F6D1226802F108038E
:107C200053E8003F23F00103083242E80031002905
:107C3000F3D12023C4F88C30002384F8843003204F
:107C4000B7E778B310B50446D0F888300BB32423D7
:107C5000C4F888302268136823F001031360A36A14
:107C6000E3B92046FFF76CFB012811D02268536866
:107C700023F4904353602268936823F02A039360AF
:107C80002268136843F0010313602046FFF774FF76
:107C900010BD80F88430FAF7ABF9D8E72046FFF73B
:107CA000B3FEDEE701207047436E2BB90123A0F835
:107CB0006A30A0F86830704730B403689A68C2F33D
:107CC00042629968490F094D6B5C1B01084C615C6D
:107CD00093FBF1F3A0F86A30AB5C1B01A25C93FB51
:107CE000F2F3A0F8683030BC704700BF1CB6000843
:107CF00014B6000870477047704790F88430012B25
:107D000018D0012380F884302423C0F88830036819
:107D10001A68196821F00101196022F0005200234D
:107D2000436601680A602022C0F8882080F8843009
:107D3000184670470220704738B590F88430012B00
:107D40001DD00446012380F884302423C0F88830F5
:107D500003681D681A6822F001021A6002689368BD
:107D600023F0604319439160FFF79EFF23681D6075
:107D70002023C4F88830002084F8840038BD022015
:107D8000FCE738B590F88430012B1DD00446012360
:107D900080F884302423C0F8883003681D681A688E
:107DA00022F001021A600268936823F060631943AD
:107DB0009160FFF779FF23681D602023C4F88830A5
:107DC000002084F8840038BD0220FCE72DE9F04F44
:107DD00085B08346019103920023029331E007EBC3
:107DE000C506D6E900890BEB0A0101EBC401019B32
:107DF00003EB441303EBC503D3E90023D1E90001EE
:107E0000F8F742FC02460B4640464946F8F786FA28
:107E1000C6E900010134032CE1DD0135032D0DDC41
:107E2000029B4FEA431A039A02EB431707EBC50381
:107E300000200021C3E900010024ECE7029B01338C
:107E40000293029B032B01DC0025E7E705B0BDE8A8
:107E5000F08F000010B4034610464C1EA4B231B19E
:107E600013F8011B4140034A505C2146F5E710BC62
:107E7000704700BF24B60008034690B1481E91B178
:107E800010B413F8011B5140C9B2084C34F811105A
:107E900081EA1222014601380029F2D1104610BCB5
:107EA00070474FF6FF721046704700BF24B70008B6
:107EB000F8B53B4C4FF488752A460021204601F066
:107EC00049F82A460021601901F044F82A460021A9
:107ED00004F5087001F03EF82A46002104F54C70C4
:107EE00001F038F82A46002104F5886001F032F8E4
:107EF0002A46002104F5AA6001F02CF80123238012
:107F00000522628084F8583084F83C30254A226487
:107F10004FF07E562665244D65652448C4F8B000B0
:107F20002349C4F8B410234AC4F8B8200227A4F89F
:107F300010710627A4F8127184F8683184F84C3166
:107F4000C4F86061C4F86451C4F8C001C4F8C41135
:107F5000C4F8C8210327A4F820720727A4F82272C6
:107F600084F8783284F85C32C4F87062C4F87452D1
:107F7000C4F8D002C4F8D412C4F8D8220425A4F856
:107F800030530825A4F8325384F8883384F86C33CE
:107F9000C4F8E003C4F8E413C4F8E823F8BD00BF54
:107FA000BC0600249A99D9BFCDCC4C3E0000484174
:107FB0000000F0410000204108B590F85830013B26
:107FC0002C2B32D8DFE813F02D00320037003C00B4
:107FD000410046004B00500055005A005F0064000D
:107FE00069006E00730078007D00820087008C00BD
:107FF000910096009B00A000A500AA00AF00B4006D
:10800000B900BE00C300C800CD00D200D700DC001C
:10801000E100E600EB00F000F500FA00FF000401CB
:1080200009010021008800F05DFC08BD01210088E5
:1080300000F058FCF9E70221008800F053FCF4E757
:108040000321008800F04EFCEFE70421008800F0D7
:1080500049FCEAE70521008800F044FCE5E7062139
:10806000008800F03FFCE0E70721008800F03AFCC0
:10807000DBE70821008800F035FCD6E709210088FD
:1080800000F030FCD1E70A21008800F02BFCCCE79F
:108090000B21008800F026FCC7E70C21008800F0C7
:1080A00021FCC2E70D21008800F01CFCBDE70E2179
:1080B000008800F017FCB8E70F21008800F012FCE0
:1080C000B3E71021008800F00DFCAEE71121008815
:1080D00000F008FCA9E71221008800F003FCA4E7E7
:1080E0001321008800F0FEFB9FE71421008800F0B8
:1080F000F9FB9AE71521008800F0F4FB95E71621BB
:10810000008800F0EFFB90E71721008800F0EAFB01
:108110008BE71821008800F0E5FB86E7192100882D
:1081200000F0E0FB81E71A21008800F0DBFB7CE730
:108130001B21008800F0D6FB77E71C21008800F0A7
:10814000D1FB72E71D21008800F0CCFB6DE71E21FA
:10815000008800F0C7FB68E71F21008800F0C2FB21
:1081600063E72021008800F0BDFB5EE72121008845
:1081700000F0B8FB59E72221008800F0B3FB54E778
:108180002321008800F0AEFB4FE72421008800F097
:10819000A9FB4AE73221008800F0A4FB45E7332120
:1081A000008800F09FFB40E73421008800F09AFB34
:1081B0003BE73521008800F095FB36E73621008843
:1081C00000F090FB31E73721008800F08BFB2CE7B3
:1081D0005021008800F086FB27E75121008800F03D
:1081E00081FB22E790F8583013B18B78332B00D005
:1081F000704710B4CA780C79002364F307034C79F4
:1082000064F30F238C7964F31743C97961F31F6317
:10821000512A57D8DFE812F0520058005D00620082
:1082200067006C00710076007B00800086008C0087
:10823000920098009E00A400AA00B000B600BC0006
:10824000C200C800CE00D400DA00E000E600EC0076
:10825000F200F800FE0004010A01100116011C01E1
:108260002201560056005600560056005600560091
:1082700056005600560056005600560028012E01A2
:1082800034013A014001460156005600560056009E
:10829000560056005600560056005600560056002E
:1082A000560056005600560056005600560056001E
:1082B00056005600560056004C015201C365022379
:1082C00080F8583010BC70470366032380F858309C
:1082D000F8E74366042380F85830F3E78366052304
:1082E00080F85830EEE7C366062380F85830E9E797
:1082F0000367072380F85830E4E74367082380F8D2
:108300005830DFE78367092380F85830DAE7C3671E
:108310000A2380F85830D5E7C0F880300B2380F866
:108320005830CFE7C0F884300C2380F85830C9E7C4
:10833000C0F888300D2380F85830C3E7C0F88C307F
:108340000E2380F85830BDE7C0F890300F2380F836
:108350005830B7E7C0F89430102380F85830B1E7B0
:10836000C0F89830112380F85830ABE7C0F89C3043
:10837000122380F85830A5E7C0F8A030132380F806
:1083800058309FE7C0F8A430142380F8583099E79C
:10839000C0F8A830152380F8583093E7C0F8AC3007
:1083A000162380F858308DE7C0F8B030172380F8D6
:1083B000583087E7C0F8B430182380F8583081E788
:1083C000C0F8B830192380F858307BE7C0F8BC30CB
:1083D0001A2380F8583075E7C0F8C0301B2380F8A6
:1083E00058306FE7C0F8C4301C2380F8583069E774
:1083F000C0F8C8301D2380F8583063E7C0F8CC308F
:108400001E2380F858305DE7C0F8D0301F2380F875
:10841000583057E7C0F8D430202380F8583051E75F
:10842000C0F8D830212380F858304BE7C0F8DC3052
:10843000222380F8583045E7C0F8E030232380F845
:1084400058303FE7C0F8E430242380F8583039E74B
:10845000C0F8E830252380F8583033E7C0F8EC3016
:10846000262380F858302DE7C0F8F030272380F815
:10847000583027E7C0F8F430282380F8583021E737
:10848000C0F8F830292380F858301BE7C0F8FC30DA
:108490002A2380F8583015E7C0F800312B2380F8E4
:1084A00058300FE7C0F804312C2380F8583009E722
:1084B000C0F808312D2380F8583003E7C0F80C319C
:1084C000002380F85830FDE610B584B000230193F6
:1084D000029301AA0DF10E011A48F9F79FF9BDF8B0
:1084E0000E30053B032B0CD8DFE803F0020D1721FB
:1084F000154C01A9204600F067F801A92046FFF7B6
:1085000071FE04B010BD114C01A9204600F05CF8CA
:1085100001A92046FFF766FEF3E70D4C01A92046AE
:1085200000F052F801A92046FFF75CFEE9E7094C8C
:1085300001A9204600F048F801A92046FFF752FEA5
:10854000DFE700BF74040024BC060024CC0700242D
:10855000DC080024EC090024F8B505460F461E4649
:108560001046F8F77FFB044639462846F8F77AFBB1
:1085700005460120B0400138F8F72AFC014628469C
:10858000F8F77AFC2146F8F72BFDF8F7C5FDF8BDA2
:10859000F8B507460C461E461046F8F763FB05463D
:1085A0003846F8F715FC2946F8F766FC0546012021
:1085B000B0400138F8F70CFC01462846F8F710FDEA
:1085C0002146F8F751FBF8BDF8B504460D460B7887
:1085D00003F00F0343600B781B0983604B788878A6
:1085E00040EA0320E060CB780F793F0947EA0317A0
:1085F00027610E79360206F470664B791E43666178
:10860000D4F8B02002F100411023FFF7C1FF20622F
:10861000D4F8B42002F100410C233846FFF7B8FF2C
:108620006062D4F8B82002F100410C233046FFF715
:10863000AFFFA062A879F8F7C7FB6063E879F8F7A5
:10864000C3FBA063F8BD00B583B01144FF238DF8D0
:1086500000308DF801308DF802308DF803308DF840
:1086600004308DF805308DF80630FC238DF8073086
:1086700008236A4689B2F9F792F803B05DF804FB63
:1086800008B591F83C30013B032B07D8DFE803F035
:1086900002070D1300220988FFF7D5FF08BD4FF42C
:1086A00080720988FFF7CFFFF8E74FF4007209885E
:1086B000FFF7C9FFF2E74FF440720988FFF7C3FFE5
:1086C000ECE700002DE9F04F87B002900C460392D2
:1086D0001846D1F8B02002F100411023FFF73CFF0B
:1086E0000190BDF80480D4F8B42002F100410C23BD
:1086F0001098FFF731FF064687B2D4F8B82002F190
:1087000000410C231398FFF727FF05461FFA80FA54
:108710004FF000090C231B4A49461198FFF71CFF34
:1087200004461FFA80FB0C23174A49461298FFF7AC
:1087300013FF4FEA18288DF81080019B8DF8113037
:108740003F098DF81270114B03EA061242EA1B2B07
:108750008DF813B08DF81440C0F30B128DF815206E
:1087600003EA001343EA1A2A8DF816A08DF8175071
:10877000082304AA03990298F9F711F807B0BDE895
:10878000F08F00BF0000FA430000A040F0FF0F0090
:1087900010B582B001F580718DF80020C2F3072476
:1087A0008DF80140C2F307448DF80240C2F307621E
:1087B0008DF803208DF80430C3F307228DF80520CF
:1087C000C3F307428DF80620C3F307638DF8073023
:1087D00008236A4689B2F8F7E2FF02B010BD00B57F
:1087E00083B001F500718DF80420C2F307238DF8E2
:1087F0000530C2F307438DF80630C2F307628DF8E7
:10880000072004230DEB030289B2F8F7C8FF03B079
:108810005DF804FBF0B583B007460E4614461849D0
:108820001846F8F729FBF8F79DFC85B2154908981A
:10883000F8F722FBF8F796FC06F540718DF800403A
:10884000C4F307238DF80130C4F307438DF80230D9
:10885000C4F307628DF803208DF80450C5F3072593
:108860008DF805508DF80600C0F307208DF807003D
:1088700008236A4689B23846F8F791FF03B0F0BD85
:108880000000C84200401C4600B585B091F83C305D
:10889000013B032B0FD8DFE803F00211171C8B6C90
:1088A00003934B6D02930B6D01934B6C00930B6C18
:1088B0000A88FFF707FF05B05DF804FB4B6C0A6CF4
:1088C0000988FFF765FFF6E74A6C0988FFF787FF1D
:1088D000F1E7CB6C00934B6C0A6C0988FFF79AFFA9
:1088E000E9E7000000B583B000F00F03C0F3031008
:1088F0008DF804308DF8050033238DF806308DF89F
:10890000071004230DEB030240F2FF710248F8F751
:1089100046FF03B05DF804FB74040024000000006F
:10892000F0B4234B00200021C3E90201C3E92E016A
:10893000C3E95A0112A5D5E90045C3E9864512A548
:10894000D5E90045C3E9004511A5D5E90045C3E9CE
:108950002C45C3E9580110A5D5E90045C3E9844574
:108960000FA5D5E90045C3E904450FA7D7E900677E
:10897000C3E93067C3E95C45C3E98801F0BC7047CF
:108980003BDF4F8D976EA23FDBF97E6ABC74B33F2D
:108990001904560E2DB2BD3FFA7E6ABC7493C03FD7
:1089A0007A008BFCFA21F9BF7A008BFCFA21F93F9F
:1089B000601100242DE9F04F87B00E4D286AF7F7BB
:1089C0000BFE0D4CC4E90601D5F83001F7F704FEA3
:1089D000C4E93201D5F84002F7F7FEFDC4E95E01B3
:1089E000D5F85003F7F7F8FDC4E98A014FF0000B02
:1089F0007AE000BFBC06002460110024C24BB02402
:108A000004FB0B34D4E906894046494600F062FB7A
:108A10008A46029002460B46C4E90C23404649466A
:108A200000F0AEFB00900D4601F100430493D4E941
:108A300004894046494600F04DFB06460F46024673
:108A40000B4600980499F7F71FFEC4E90E01404653
:108A5000494600F095FB8046894602460B46009841
:108A60002946F7F711FEC4E91001D4E90223CDE944
:108A7000042302985146F7F707FEC4E91201009A51
:108A80002B46C4E9142332463B4602985146F7F779
:108A9000FBFDC4E91601029A0AF10043404649462B
:108AA000F7F7F2FDC4E91801DDE90423009829462F
:108AB000F7F7EAFDC4E91A0100200021C4E91C010E
:108AC000C4E91E89C4E92067D4E90023C4E922234C
:108AD000C4E92401C4E92601C4E9280100228B4B22
:108AE000C4E92A230BF1010BBBF1030F86DD884D8E
:108AF000DFF814A22A460AF1E0010AF13000FFF77C
:108B000065F9844C22460AF5C8712846FFF75EF9DC
:108B1000DFF804B25A460AF510712046FFF756F9FD
:108B2000DBE90E45DAE98667DBE90823304639469A
:108B3000F7F7AAFD02460B4620462946F7F7ECFB5D
:108B400080468946DAE98445DBE90C23204629463C
:108B5000F7F79AFD02460B4640464946F7F7DCFB1D
:108B6000CDE90001DBE90689DBE90023304639461F
:108B7000F7F78AFD02460B4640464946F7F7CCFB1D
:108B800006460F46DBE9042320462946F7F77CFD1D
:108B900002460B4630463946F7F7BEFB02460B4607
:108BA000DDE9000100F0A0FB04460D460022002391
:108BB000DAE92C0100F098FB02460B4620462946D4
:108BC000F7F7AAFB02460B46CAE90823DBE90C4586
:108BD00000F080FA02460B4620462946F7F754FD7E
:108BE00004460D46DBE90467DAE9060100F0C8FA3D
:108BF00002460B4630463946F7F746FD02460B461D
:108C000020462946F7F788FB00F012FBCAE960010D
:108C1000DBE90C45DAE9080100F05CFA02460B4694
:108C200020462946F7F730FD04460D46DBE9046788
:108C3000DAE9060100F0A4FA02460B46304639464E
:108C4000F7F722FD02460B4620462946F7F764FB5C
:108C500000F0EEFA024601F10043CAE96223DBF8B4
:108C60003040DBF8346006F10045DBE90489424618
:108C70004B462046294600F037FBCDE90201DAE9F0
:108C8000340100F027FACDE90001224633462046A0
:108C90003146F7F7F9FC06460F4642464B4640463A
:108CA0004946F7F7F1FC02460B4630463946F7F7DE
:108CB00035FB06460F46DDE9000102460B46F7F795
:108CC000E3FC02460B4630463946F7F725FB00F039
:108CD0000DFB02460B46DDE9000100F005FB0246F4
:108CE0000B46DDE90201F7F717FBCAE98E014246A0
:108CF0004B462046294600F0F7FA80468946DAE9D5
:108D0000344520460AE000BF601100240000F03F17
:108D100020140024A014002420150024294600F06B
:108D20002FFACDE900012046294600F0D3F902468A
:108D30000B46F7F7A9FC02460B4630463946F7F7D3
:108D4000EBFA00F0D3FA024601F10043DDE900013D
:108D500000F0CAFA02460B4640464946F7F7DCFAED
:108D6000CAE98C01DBE91445DAE9600100F008FA90
:108D700002460B4620462946F7F7B0FD00F086FA7A
:108D8000CAE93401DBE91445DAE9600100F0F8F9D9
:108D900002460B4620462946F7F7A0FD00F076FA7A
:108DA000054601F1004402462346CAE93623DAE9C2
:108DB0000801F7F703FF2C4B1864DAE95E6700221D
:108DC000002330463946F7F7E5FE00283AD0DAE9C5
:108DD0003401F7F7F3FE244BC3F8500100220023BF
:108DE00030463946F7F7D6FE002833D01F4BD3E97B
:108DF0006001F7F7E3FE1C4BC3F860021B4DD5E999
:108E00008C01F7F7DBFE184CC4F87003D5E90601B6
:108E100000F0B6F9164BD3E90023F7F735FCF7F766
:108E2000CDFEA0643046394600F0AAF9114BD3E9D3
:108E30000023F7F729FCF7F7C1FEC4F8680207B072
:108E4000BDE8F08F28462146F7F7B8FE064BC3F879
:108E50005001C3E7054BD3E96201F7F7AFFE024BC0
:108E6000C3F86002CAE700BFBC06002460110024FA
:108E7000100000241800002410B5094CA52323700D
:108E800000231E226270A370E370FF22042120469B
:108E9000FEF7E0FF2071022363710323A37110BD6D
:108EA000A415002438B5134C134D2B78E370FF2222
:108EB00004212046FEF7CEFF2071104B9A89A4F8BA
:108EC0000720B3F81C21A4F80920B3F82C22A4F839
:108ED0000B20B3F83C33A4F80D304FF6FF72252178
:108EE0002046FEF7C9FFA4F825002B7801332B702C
:108EF00038BD00BFA4150024A0150024BC06002422
:108F0000014B1868704700BF2000002470B50D4E5B
:108F10000D4D761BB61006D0002455F8043B0134E5
:108F20009847A642F9D1094E094D761B02F01EFB67
:108F3000B61006D0002455F8043B01349847A642E9
:108F4000F9D170BD80BB000880BB000888BB000859
:108F500080BB0008F0B4860746D0541E002A3CD0DF
:108F6000CAB2034601E0013C37D303F8012B9D0749
:108F7000F9D1032C2AD9CDB245EA05250F2C45EAB3
:108F8000054534D9A4F1100222F00F0C03F120079B
:108F90001609674403F1100242E9045542E90255FB
:108FA0001032BA42F8D1721C14F00C0F03EB02120B
:108FB00004F00F0613D0331F23F0030304331344CC
:108FC00042F8045B9342FBD106F003042CB1CAB211
:108FD0001C4403F8012B9C42FBD1F0BC7047344683
:108FE0001346002CF3D1F8E714460346C1E71A46AE
:108FF0002646E0E7024B13B1024800F005B870477F
:109000000000000015900008002301461A4618468B
:1090100000F01AB838B5084B084D5B1B9C1007D000
:10902000043B1D44013C55F804399847002CF9D104
:10903000BDE8384002F0A0BA8CBB000888BB00082D
:10904000704700BF704700BF2DE9F047DFF880A0F0
:109050000646DAF8000098460F469146FFF7F0FF03
:109060001A4B1B68D3F8484124B365681F2D26DCD2
:109070005EB9AB1C0135DAF80000656044F8237076
:10908000FFF7E0FF0020BDE8F08704EB8503012136
:10909000C3F88890D4F88821A9400A43022EC4F866
:1090A0008821C3F80881E4D1D4F88C311943C4F87D
:1090B0008C11DEE703F5A674C3F84841D5E7DAF86A
:1090C0000000FFF7BFFF4FF0FF30DCE724B90008D6
:1090D00050040024F0B5284D21F00043AB4287B086
:1090E00021DD264DAB4209DD02460B46F7F714F9A8
:1090F00002460B461046194607B0F0BD02AA00F022
:1091000087FE00F00300012817D0022829D0F8B10B
:1091100001230093DDE90201DDE9042301F0B4FE3F
:109120000B460246E6E70022002301F059F90B4600
:1091300002461046194607B0F0BDDDE90423009051
:10914000DDE9020101F0A0FE024601F10043D1E792
:10915000DDE90423DDE9020101F042F90B46024694
:10916000C8E7DDE90423DDE9020101F039F902462F
:1091700001F10043BEE700BFFB21E93FFFFFEF7FA6
:10918000F0B5294D21F00043AB4287B020DD274DDB
:10919000AB4209DD02460B46F7F7BEF802460B4626
:1091A0001046194607B0F0BD02AA00F031FE00F0EB
:1091B0000300012818D002282AD0F0B1DDE90423E9
:1091C000DDE9020101F00CF9024601F10043E7E795
:1091D000002300930022002301F056FE0B460246B6
:1091E0001046194607B0F0BDDDE90423DDE90201B0
:1091F00001F0F6F80B460246D2E701230093DDE9C1
:109200000201DDE9042301F03FFE0B460246C7E7F9
:1092100001230093DDE90201DDE9042301F034FEBE
:10922000024601F10043BBE7FB21E93FFFFFEF7F6F
:10923000F8B504460D4600F087F8114B93F900305D
:10924000013306460F460FD022462B4620462946BC
:10925000F8F7BCF940B92046294602F083F8094BDB
:109260000022F7F7A1FC10B930463946F8BDFFF7E8
:1092700047FE21230360BDE8F840034802F0F4B83C
:10928000540400240000F03F28B90008F8B5044653
:109290000D4600F0ADFA114B93F90030013306464C
:1092A0000F460FD022462B4620462946F8F78EF966
:1092B00040B92046294602F055F8094B0022F7F73D
:1092C00073FC10B930463946F8BDFFF719FE21236B
:1092D0000360BDE8F840034802F0C6B85404002417
:1092E0000000F03F28B9000800F0C6BCF8B50446FD
:1092F0000D4600F0AFFF134B93F9003001330646E3
:109300000F460DD022462B4620462946F8F75EF937
:1093100030B92046294600220023F7F727FC10B970
:1093200030463946F8BDFFF7EBFD0022002321212E
:10933000016010461946F7F7D1FA06460F46304647
:109340003946F8BD540400242DE9F84FC44F21F0EC
:10935000004CBC450C4605460DDD0CF1404303F5C1
:109360008013034340F0B980002940F3C0800020FF
:109370000021BDE8F88FBB4A944508DCBA4A944501
:1093800000F3BA809CA1D1E90001BDE8F88F002963
:10939000C0F2708102460B460020B449F6F7BCFFCC
:1093A000B34B0022F7F770F904460D4600F052FF68
:1093B00093A3D3E900238946804629462046F7F740
:1093C00063F991A3D3E90023F6F7A8FF22462B46C1
:1093D000F7F75AF98EA3D3E90023F6F79DFF22464B
:1093E0002B46F7F751F98CA3D3E90023F6F796FF44
:1093F00022462B46F7F748F989A3D3E90023F6F76D
:109400008BFF22462B46F7F73FF987A3D3E90023CA
:10941000F6F784FF22462B46F7F736F984A3D3E903
:10942000002382468B4620462946F7F72DF982A372
:10943000D3E90023F6F770FF22462B46F7F724F90D
:109440007FA3D3E90023F6F769FF22462B46F7F7FF
:109450001BF97DA3D3E90023F6F75EFF22462B46D6
:10946000F7F712F9814B0022F6F758FF02460B4638
:1094700050465946F7F732FA42464B46F7F704F999
:10948000002682468B4632464B4630464946F7F721
:10949000FBF802460B4620462946F6F73DFF3246CA
:1094A00004460D464B4640464946F6F737FF02460E
:1094B0000B4620462946F7F711FA02460B4650465E
:1094C0005946F6F72BFF32464B46F6F727FF024682
:1094D0000B46F6F723FFBDE8F88F02460B46F6F77A
:1094E0001BFF02460B46F7F7F9F9BDE8F88F58A1C4
:1094F000D1E90001BDE8F88F02460B46F7F7C4F842
:109500003FA3D3E9002306460F46F7F7BDF83EA375
:10951000D3E90023F6F702FF32463B46F7F7B4F8EB
:109520003BA3D3E90023F6F7F7FE32463B46F7F7B5
:10953000ABF839A3D3E90023F6F7F0FE32463B46F9
:10954000F7F7A2F836A3D3E90023F6F7E5FE324693
:109550003B46F7F799F834A3D3E90023F6F7DEFE8C
:1095600032463B46F7F790F831A3D3E90023804613
:10957000894630463946F7F787F82FA3D3E9002309
:10958000F6F7CAFE32463B46F7F77EF82CA3D3E93E
:109590000023F6F7C3FE32463B46F7F775F82AA3D9
:1095A000D3E90023F6F7B8FE32463B46F7F76CF8EE
:1095B0002E4B0022F6F7B2FE02460B4640464946C5
:1095C000F7F78CF92A462346F7F75EF802460B4672
:1095D00021A1D1E90001F6F79FFE02460B4628467D
:1095E0002146F6F799FE02460B4603A1D1E9000198
:1095F000F6F792FEBDE8F88F182D4454FB21F93F91
:1096000009F7FD0DE13D023F88B20175E0EF493FEA
:109610003B8F68B52882A43F5544880E55C1C93F89
:109620007D6FEB0312D6D43F555555555555C53F63
:1096300082922EB1C5B8B33F59018D1B6C06E63F2F
:10964000C88A599CE52A00404B2D8A1C273A0340C2
:10965000182D4454FB210940075C143326A6913C85
:10966000FFFFEF3FFFFFDF3F0000603C0000F03FE7
:109670000000E03F5C4B0022F6F750FE5B4B0022FF
:10968000F7F702F840A3D3E9002304460D46F6F7A6
:10969000FBFF3FA3D3E90023F6F740FE22462B460B
:1096A000F6F7F2FF3CA3D3E90023F6F735FE224696
:1096B0002B46F6F7E9FF3AA3D3E90023F6F72EFE8F
:1096C00022462B46F6F7E0FF37A3D3E90023F6F74F
:1096D00023FE22462B46F6F7D7FF35A3D3E9002316
:1096E000F6F71CFE22462B46F6F7CEFF804689464B
:1096F0002046294600F0AEFD2FA3D3E900230646FD
:109700000F4620462946F6F7BFFF2DA3D3E90023D5
:10971000F6F702FE22462B46F6F7B6FF2AA3D3E958
:109720000023F6F7FBFD22462B46F6F7ADFF28A3F4
:10973000D3E90023F6F7F0FD22462B46F6F7A4FF07
:10974000294B0022F6F7EAFD02460B464046494601
:10975000F7F7C4F832463B46F6F796FF1EA3D3E967
:109760000023F6F7D9FD32463B46F6F7D7FD024611
:109770000B46F6F7D3FD02460B4619A1D1E90001CD
:10978000F6F7CAFDBDE8F88F09F7FD0DE13D023F90
:1097900088B20175E0EF493F3B8F68B52882A43F4E
:1097A0005544880E55C1C93F7D6FEB0312D6D43F97
:1097B000555555555555C53F82922EB1C5B8B33F45
:1097C00059018D1B6C06E63FC88A599CE52A00406A
:1097D0004B2D8A1C273A0340075C143326A6913C84
:1097E000182D4454FB2109400000F03F0000E03FE9
:1097F0002DE9F04FCA4B21F000479F4287B00C463D
:10980000054616DD07F1404707F5801703463B4341
:1098100000F00C8102460B46F6F77EFD02460B4631
:10982000F7F75CF803460A461846114607B0BDE84C
:10983000F08FBC4B9F420E460FDCB7F1795F80F290
:1098400079819BA3D3E90023F6F768FDB64B00228C
:10985000F7F7AAF9002840F027812846214601F0B1
:1098600081FD02460B460020AF49F6F755FDAF4B90
:109870000022F6F709FF90A3D3E9002304460D4622
:10988000F6F702FF8EA3D3E90023F6F747FD224641
:109890002B46F6F7F9FE8CA3D3E90023F6F73CFD3F
:1098A00022462B46F6F7F0FE89A3D3E90023F6F70C
:1098B00035FD22462B46F6F7E7FE87A3D3E90023C2
:1098C000F6F72AFD22462B46F6F7DEFE84A3D3E9FF
:1098D0000023F6F723FD22462B46F6F7D5FE82A39A
:1098E000D3E900238046894620462946CDE90289EE
:1098F000F6F7CAFE7EA3D3E90023F6F70DFD224654
:109900002B46F6F7C1FE7CA3D3E90023F6F706FD4C
:1099100022462B46F6F7B8FE79A3D3E90023F6F7E3
:10992000FBFC22462B46F6F7AFFE7F4B0022F6F7F4
:10993000F5FC02460B4692469B4620462946CDE959
:1099400004AB00F087FCDFF8E8C167458046894634
:1099500000F389808B464FF0000A02460B46CDE9A2
:1099600000ABF6F7DBFCDDE9042382468B46DDE93C
:109970000201F6F7B3FF02460B4650465946F6F78A
:1099800083FEDDE9002382468B4610461946F6F732
:109990007BFE02460B4620462946F6F7BDFCDDE974
:1099A000002304460D4640464946F6F7B7FC0246FA
:1099B0000B4620462946F6F791FF02460B46F6F77E
:1099C000ADFC02460B4650A1D1E90001F6F7A4FC1C
:1099D00002460B4650465946F6F79EFCDDE9002349
:1099E00004460D4610461946F6F798FC02460B460B
:1099F00047A1D1E90001F6F78FFC02460B4620464D
:109A00002946F6F789FC02460B4641A1D1E900013F
:109A1000F6F782FC03460A46002E3FF705AF02F137
:109A200000421846114607B0BDE8F08F3AA3D3E9CB
:109A30000023F6F729FE02460B46284621461D461E
:109A4000144631A3D3E90023F6F71EFE02460B4667
:109A500020462946F6F762FC03460A461846114698
:109A600007B0BDE8F08F52465B46DDE90201F6F72C
:109A700035FF42464B46F6F707FE42464B46F6F7A1
:109A80004DFC02460B46F6F749FC1FA3D3E9002321
:109A9000F6F742FC02460B461FA1D1E90001F6F79A
:109AA0003BFC03460A46B7E72B462246BCE600BF0E
:109AB0009C7500883CE4377E09F7FD0DE13D023FCF
:109AC00088B20175E0EF493F3B8F68B52882A43F1B
:109AD0005544880E55C1C93F7D6FEB0312D6D43F64
:109AE000555555555555C53F82922EB1C5B8B33F12
:109AF00059018D1B6C06E63FC88A599CE52A004037
:109B00004B2D8A1C273A0340075C143326A6913C50
:109B1000182D4454FB21E93F182D4454FB21F93FF3
:109B2000FFFFEF3FFFFFDF3F0000F03F0000E03F9F
:109B30003233EF3F02460B46F6F7A6FD38A3D3E9D2
:109B4000002306460F46F6F79FFD37A3D3E900230F
:109B5000F6F7E4FB32463B46F6F796FD34A3D3E92D
:109B60000023F6F7D9FB32463B46F6F78DFD32A3CC
:109B7000D3E90023F6F7D2FB32463B46F6F784FDE5
:109B80002FA3D3E90023F6F7C7FB32463B46F6F78F
:109B90007BFD2DA3D3E90023F6F7C0FB32463B46FD
:109BA000F6F772FD2AA3D3E90023804689463046A2
:109BB0003946F6F769FD28A3D3E90023F6F7ACFB95
:109BC00032463B46F6F760FD25A3D3E90023F6F7BE
:109BD000A5FB32463B46F6F757FD23A3D3E9002306
:109BE000F6F79AFB32463B46F6F74EFD204B002235
:109BF000F6F794FB02460B4640464946F6F76EFEE2
:109C00002A462346F6F740FD2A462346F6F786FB0A
:109C100003460A461846114607B0BDE8F08F00BF5C
:109C200009F7FD0DE13D023F88B20175E0EF493FC4
:109C30003B8F68B52882A43F5544880E55C1C93F63
:109C40007D6FEB0312D6D43F555555555555C53F3D
:109C500082922EB1C5B8B33F59018D1B6C06E63F09
:109C6000C88A599CE52A00404B2D8A1C273A03409C
:109C70000000F03F000000002DE9F84F1F4653425E
:109C80005F4E134327F0004949EAD373B342944629
:109C90000D4686463BD84442044321F0004A4AEA36
:109CA000D474B44203468B4631D807F1404404F5DE
:109CB000801414433BD0BC1704F002045AEA030397
:109CC00044EAD1742BD059EA020334D0B14545D0CF
:109CD000B24530D0AAEB0909B9F1747F4FEA295394
:109CE00038DA002F46DA3C3344DA00200021012C18
:109CF00058D0022C49D084B135A3D3E90023F6F71C
:109D00000BFB35A3D3E90023F6F706FB05E072460B
:109D100060462B463946F6F701FBBDE8F88F022C6A
:109D200010D0032CF9D12EA1D1E90001F5E7BDE84F
:109D3000F84F01F06DB9BBF1000F07DB2AA1D1E9A3
:109D40000001EAE724A1D1E90001E6E728A1D1E971
:109D50000001E2E724A1D1E90001C8E7CA4504F106
:109D6000FF3423D0022C29D8264B03EBC404D4E9BA
:109D70000001D2E7624670463B462946F6F7AEFD43
:109D800001F0F0FA01F044F9B1E711A3D3E900239F
:109D9000F6F7C2FA02460B460FA1D1E90001F6F729
:109DA000BBFABAE701F100431946B6E7022C08D81E
:109DB000154B03EBC404D4E90001AEE700200021F9
:109DC000ABE70DA1D1E90001A7E700BFAFF3008029
:109DD000075C143326A6A13C182D4454FB210940EE
:109DE000182D4454FB2109C0182D4454FB21F93F80
:109DF000182D4454FB21F9BF182D4454FB21E93F91
:109E00000000F07F48B9000830B9000800000000E9
:109E10002DE9F04F8C4F21F00045BD428DB0144626
:109E2000064640F38680894A95428B4627DC002906
:109E30007BA3D3E9002340F3B881F6F76DFA844B96
:109E40009D4206460F4600F08B8077A3D3E900239E
:109E5000F6F762FA02460B46C4E90023304639465B
:109E6000F6F75AFA70A3D3E90023F6F755FAC4E9D6
:109E700002014FF0010A50460DB0BDE8F08F754A5F
:109E8000954240F38E80744A95425EDC4FEA255A33
:109E9000AAF2164AA5EB0A510F46F7F7ADFBF6F703
:109EA00089FB804689463046394642464B46CDE9D5
:109EB0000689F6F731FA694B0022F6F7E5FB0F4603
:109EC0000646F7F799FB0546F6F774FB02460B4684
:109ED00030463946CDE90823F6F71EFA5F4B0022DB
:109EE000F6F7D2FB02460B46CDE90A2300220023F7
:109EF000F6F732FE002800F05681002D0CBF01233A
:109F00000223574A019202215246009106A8214697
:109F100000F092FBBBF1000F8246ACDA6268E368A6
:109F200002F1004203F10043C0F1000A6260E36005
:109F3000A1E74FF0000AC4E90001002200235046C7
:109F4000C4E902230DB0BDE8F08F02465B46F6F788
:109F5000E3F94FF0000AC4E90201C4E900018AE70D
:109F600033A3D3E90023F6F7D7F933A3D3E90023CA
:109F700006460F46F6F7D0F902460B46C4E9002321
:109F800030463946F6F7C8F92BA3D3E90023F6F794
:109F9000C3F94FF0010AC4E9020150460DB0BDE813
:109FA000F08F01F0DFF926A3D3E9002306460F4620
:109FB000F6F76AFB2B4B0022F6F7B0F9F7F71CFB1C
:109FC0008246F6F7F7FA16A3D3E9002380468946BE
:109FD000CDE90489F6F758FB02460B463046394670
:109FE000F6F79AF906460F4640464946B046B94646
:109FF0000DA3D3E90023CDE90289F6F745FBBAF1B9
:10A000001F0F06460F4631DC174B0AF1FF3253F89B
:10A010002230AB422AD002460B46404649469EE0DB
:10A0200000004054FB21F93F3163621A61B4D03D16
:10A030000000601A61B4D03D7370032E8A19A33BEF
:10A0400083C8C96D305FE43FFB21E93F7BD9024003
:10A05000FB21F93FFB213941FFFFEF7F00007041F9
:10A06000E0B900080000E03F60B900083B46DDE9C8
:10A0700002013246F6F750F9C1F30A53C3EB155308
:10A08000102B894680464FEA25556CDD66A3D3E93F
:10A090000023DDE90401F6F7F7FA06460F4602460B
:10A0A0000B46DDE90201F6F737F98046894642465C
:10A0B0004B46DDE90201F6F72FF932463B46F6F74B
:10A0C0002BF95BA3D3E9002306460F46DDE9040123
:10A0D000F6F7DAFA32463B46F6F71EF90B46024629
:10A0E00006460F4640464946CDE90289F6F714F97F
:10A0F000C1F30A53ED1A312D8946804633DD4EA354
:10A10000D3E90023DDE90401F6F7BEFADDE90256E2
:10A1100002460B468046894628463146F6F7FCF84B
:10A1200002460B4628463146CDE90223F6F7F4F8FD
:10A1300042464B46F6F7F0F841A3D3E90023064622
:10A140000F46DDE90401F6F79FFA32463B46F6F783
:10A15000E3F806460F4602460B46DDE90201F6F734
:10A16000DBF88046894642464B46C4E90023DDE9D8
:10A170000201F6F7D1F832463B46F6F7CDF8BBF1CF
:10A18000000F02460B46C4E902230546BFF673AE34
:10A1900009F1004301F10041C4E90083C4E902511F
:10A1A000CAF1000A67E60323ABE6F6F7B7F8284BD7
:10A1B0009D4206460F4616D023A3D3E90023F6F7A7
:10A1C000ADF802460B46C4E9002330463946F6F79F
:10A1D000A3F81DA3D3E90023F6F7A0F84FF0FF3A48
:10A1E000C4E9020147E610A3D3E90023F6F796F885
:10A1F0000FA3D3E9002306460F46F6F78FF8024671
:10A200000B46C4E9002330463946F6F785F808A323
:10A21000D3E90023F6F782F84FF0FF3AC4E90201D0
:10A2200029E600BFAFF300800000601A61B4D03DA2
:10A230007370032E8A19A33B0000002E8A19A33BDA
:10A24000C14920259A837B393163621A61B4D03DBC
:10A25000FB21F93F2DE9F0415F4F37EA01020E463D
:10A26000054600F0978000290B4604464EDD09158F
:10A270005AD0C3F31303CA0743F48013A1F2FF3E7D
:10A2800003D45B0003EBD4736400E20F4FF0000CC7
:10A2900002EB43034FEA6E0E6400664616254FF448
:10A2A0000012B118994202DC5B1A8E1894445B00CC
:10A2B000013D03EBD4734FEA52024FEA4404F0D15C
:10A2C0002F4620204FF0004209E03DD0E10F013839
:10A2D0004FEA520201EB43034FEA44043DD0B3423C
:10A2E00002EB0501F1DD002901EB020509DBB046B7
:10A2F0009B1BA14288BF03F1FF33641A17444646F3
:10A30000E4E7002DF3DB06F10108F1E721F000425C
:10A31000024357D000294BD1E20A15396405134690
:10A32000002AF9D0D70252D400205B00DE02054695
:10A3300000F10100F9D51A4623468440C0F12000FF
:10A34000C3401343491B94E7A142BFD8002901EB46
:10A350000205D6DB98460023CFE7234313D17808C4
:10A360004FEA6C0303F17F5303F500131CF0010F58
:10A3700018BF40F0004003EB0E5502462B46104636
:10A380001946BDE8F0817B1C16BF781C0CF1010C4E
:10A390004008E5E702460B46F6F776F92A463346CB
:10A3A000F5F7BCFF02460B4610461946BDE8F081A2
:10A3B0000246F5F7B1FF02460B46F6F78FFA024662
:10A3C0000B46DCE7024610461946BDE8F0812346FD
:10A3D00020204FF0FF35B3E70000F07F00000000C1
:10A3E0002DE9F04D21F0004786B0B7F1795FCDE956
:10A3F0000023884606466DDAF7F7FEF8002800F0DD
:10A40000EF803246434630464146F6F73DF978A3A1
:10A41000D3E9002304460D46F6F736F976A3D3E9CF
:10A420000023F5F77BFF22462B46F6F72DF974A3A0
:10A43000D3E90023F5F770FF22462B46F6F724F9FF
:10A4400071A3D3E90023F5F769FF22462B46F6F7FF
:10A450001BF96FA3D3E90023F5F75EFF22462B46D5
:10A46000F6F712F96CA3D3E90023F5F757FF22465C
:10A470002B46F6F709F9CDE90201694B0022204687
:10A480002946F6F701F9DDE9022382468B4620468C
:10A490002946F6F7F9F802460B461F463046414674
:10A4A0001646DDE90023F6F7EFF802460B46304684
:10A4B0003946F5F731FF02460B4650465946F5F747
:10A4C0002BFF02460B4600205649F5F725FF06B044
:10A4D000BDE8F08D02460B46F6F7D6F844A3D3E963
:10A4E000002304460D46F6F7CFF843A3D3E9002333
:10A4F000F5F714FF22462B46F6F7C6F840A3D3E93A
:10A500000023F5F709FF22462B46F6F7BDF83EA3D8
:10A51000D3E90023F5F702FF22462B46F6F7B4F8FD
:10A520003BA3D3E90023F5F7F7FE22462B46F6F7C7
:10A53000ABF839A3D3E90023F5F7F0FE2B4622460A
:10A54000F6F7A2F8384B9F42CDE9020195DD374B73
:10A550009F423CDC4FF0000AA7F5001B31495246F0
:10A560005B460020F5F7D8FECDE904012C4B002214
:10A5700020462946F6F788F852465B46F5F7CCFEAA
:10A58000DDE9022382468B4620462946F6F77CF811
:10A5900002460B461F46304641461646DDE900237B
:10A5A000F6F772F802460B4630463946F5F7B4FE28
:10A5B00002460B4650465946F5F7AEFE02460B469C
:10A5C000DDE90401F5F7A8FE06B0BDE8F08D184BF3
:10A5D000DFF860B00022CDE904234FF0000AC5E7A0
:10A5E0001049002006B0BDE8F08D00BFAFF3008039
:10A5F000D43888BEE9FAA8BDC4B1B4BD9EEE213EF0
:10A60000AD529C804F7E923E9015CB19A001FA3E30
:10A610007751C1166CC1563F4C5555555555A53F00
:10A620000000E03F0000F03F3233D33F0000E93F3D
:10A630000000E73F0000D23F2DE9F04FADF5197D56
:10A64000BA4CA29D089354F825400594013B12F1A1
:10A65000140F07460B910393C0F24283B449D31EF3
:10A6600081FB0301DB17C3EBA10307930133A3EBCA
:10A670008303DB00D3180693079A039BD61A059A27
:10A6800012EB03091BD409F10109DDF88CA2B144D6
:10A690000DF180080024002508E05AF82600F5F79F
:10A6A00089FF01364E45E8E8020108D0002EF4DAB1
:10A6B0000136204629464E45E8E80201F6D1059BC1
:10A6C000002BA7F108030493C0F2BA831946089B34
:10A6D000DDF80C90DA000292059A01EBC30820A97C
:10A6E00001EBC30AD3180DF5E07B0193039B002B0C
:10A6F000C0F2B181049E57460024002577E9022369
:10A70000F6E90201F5F7C0FF02460B46204629464E
:10A71000F5F704FE464504460D46EFD1019B09F1CD
:10A7200001099945EBE802450AF1080ADED1059ACC
:10A7300004980CA901EB820302990144083B8B4663
:10A740000BA90993134601EB82020A920193019A25
:10A7500098A901EBC203002A53E928452ADD0DF52B
:10A76000E07A0AEBC2080DF13009724B0022204654
:10A770002946F5F789FFF6F73FFFF5F71BFF6E4B0C
:10A78000002206460F46F5F77FFF02460B4620469D
:10A790002946F5F7C1FDF6F72FFF044678E90223B5
:10A7A00049F8044B30463946F5F7B8FDD045044624
:10A7B0000D46DAD1DDF81890204629464A4600F0C9
:10A7C0005BFE00224FF07F5304460D46F5F75CFF19
:10A7D00000F0CEFD594B0022F5F756FF02460B461E
:10A7E00020462946F5F798FD0D460446F6F704FF86
:10A7F0008046F5F7DFFE0B46024629462046F5F770
:10A800008BFD4B46002B06460F4640F39980019A7C
:10A810000CA9013AC9F1180351F8225045FA03F185
:10A8200001FA03F3EB1AC9F117050CA843FA05F571
:10A83000002D40F82230884400F38C800022002351
:10A8400030463946F6F788F9002800F05082019B1F
:10A85000059A03F1FF3A524510DC03F180430CAA3C
:10A86000013B0A9802EB8303002253F80419834248
:10A8700042EA0102F9D1002A40F0F080059B0CAABF
:10A88000013B52F82330002B40F0E080099A01236D
:10A8900052F8041901330029FAD001994A1CCB1847
:10A8A00002939146079B089902EB030A019B0B4414
:10A8B000984620AB0AF1804A03EBC808A39B0AF133
:10A8C000FF3A03EB8A0A70AB03EBC20301935AF819
:10A8D000040FF5F76FFE039B002BC8E90001474604
:10A8E00008F108081EDB049E083F0024002501E053
:10A8F00077E80201F6E90223F5F7C6FE02460B46A9
:10A9000020462946F5F70AFD5E4504460D46EFD17F
:10A91000019BE3E802450193029B09F10109994576
:10A92000D5DD13E700240025F2E700BF28BB0008AF
:10A93000ABAAAA2A0000703E00007041000020402F
:10A940006BD1019B0CAA013B52F82350ED15002D51
:10A950007FF774AF019B002B08F1010840F3C5811C
:10A960000C9C002C51D1019B012B20D00CAB01225F
:10A9700053F8044F002C4BD0531C0CA9C4F1807425
:10A9800041F822400199994210DD0CAA0CA852F816
:10A99000232000EB830300EB81006FF07F4100E098
:10A9A0001A688A1A43F8042B8342F9D10124069BC2
:10A9B000002B0EDD012B00F07A81022B09D1019BC7
:10A9C0005A1E0CAB0CA953F82230C3F3150341F8FF
:10A9D0002230022D7FF432AF32463B46BC49002084
:10A9E000F5F79AFC06460F46002C3FF427AF069A6F
:10A9F000B749002000F040FD02460B46304639467C
:10AA0000F5F78AFC06460F4618E701230022B4E753
:10AA1000019901328A42ABD1C9E7AE4B0022F6F769
:10AA2000B9F8054600283FF409AF019B002B08F157
:10AA30000108C8BF022593DC32463B46A4490020EA
:10AA4000F5F76AFC022506460F46F7E6019B5A1CFD
:10AA50009146029226E7002400255FE60CAB069A99
:10AA600053F82A30CDF81C80183A0395069273B932
:10AA7000019B03F18043023B0CA901EB830353F8D4
:10AA800004190AF1FF3A183A0029F8D00692069AFA
:10AA90008F49002000F0F0FCBAF1000F04460D468B
:10AAA000C0F2D28170AB03EBCA0B0CAA0AF101030E
:10AAB000069302EB83084FEACA030BF108090493DB
:10AAC00058F8040DF5F776FD22462B46F5F7DCFD28
:10AAD00006460F46804B2046294669E90267002258
:10AAE000F5F7D2FD0CAB984504460D46E8D148ABCE
:10AAF000CDE9013ADDF814A0BAF1000F4FF00009DA
:10AB00002CDB71A3D3E90023DFF8D0815F4600245A
:10AB10000025002603E0B14510DBF8E80223F7E842
:10AB20000201F5F7B1FD02460B4620462946F5F72E
:10AB3000F5FB0136B24504460D46ECDA019B029A5C
:10AB400003EBC9039145C3E90045ABF1080B09F1DB
:10AB5000010306D0BAF1000F9946D2DA002400258D
:10AB6000ECE7A29BDDF808A0022B23DC002B00F30E
:10AB7000F18018D1049CA29A019D08342C441346FC
:10AB80001046194674E90223F5F7C8FBA5420246B0
:10AB90000B46F5D1039909B103F1004319460B9B0C
:10ABA0001046C3E90001079B03F007000DF5197D6E
:10ABB000BDE8F08FA29B032BF5D1BAF1000F00F096
:10ABC0005981019B049A03EB020BDBE900455BE929
:10ABD00002672046294632463B46F5F79FFBA046D2
:10ABE000A94604460D4622462B4630463946F5F71F
:10ABF00093FB4B464246F5F791FBCBE900016BE92D
:10AC00000245019B5B45E2D1BAF1010F40F332816D
:10AC1000049B019A1344D3E9004502939A460DF52B
:10AC2000947B5AE902672046294632463B46F5F7AF
:10AC300075FBA046A94604460D4622462B463046E3
:10AC40003946F5F769FB42464B46F5F767FBCAE91B
:10AC500000016AE90245D345E3D1029C0199002332
:10AC600008341A4601F110051846114674E902230A
:10AC7000F5F754FBA54203460A46F5D1039900298E
:10AC800040F0B3801846019B0B9ED3E90245114664
:10AC9000DDE94823C6E90023079BC6E9040103F068
:10ACA0000700C6E902450DF5197DBDE8F08F019B4F
:10ACB0005A1E0CAB0CA953F82230C3F3160341F80B
:10ACC000223086E6AFF3008000000040FB21F93F10
:10ACD0000000F03F0000E03F0000703EF0BA0008C6
:10ACE00000216FF017030791C4E400245FE63946A2
:10ACF000069F03957A423046CDF81C8000F0BCFBDD
:10AD00005E4B002204460D46F5F744FF002862D052
:10AD10005B4B002220462946F5F7B6FCF6F76CFCA3
:10AD20000646F5F747FC554B0022F5F7ADFC0B4600
:10AD3000024629462046F5F7EFFA019CF6F75CFC3F
:10AD400004F1010A0CAB183743F82400069743F8C6
:10AD50002A609CE6019D069A002105EBC2040B4681
:10AD60000846194674E90223F5F7D8FAA5420B46BE
:10AD70000146F5D11846039B002B50D10A460C46DC
:10AD80000B9905460346C1E90045DDE94801F5F7A1
:10AD9000C3FABAF1000F02460B4610DD48AD01249C
:10ADA00010461946F5E90223F5F7B8FA0134A24531
:10ADB00002460B46F4DA039909B103F10043194640
:10ADC0000B9B1046C3E90201079B03F007000DF53A
:10ADD000197DBDE8F08F20462946F6F70DFC019B52
:10ADE0000CAA9A4642F8230051E601990B9C486848
:10ADF00023610E4602F10042B368C968A360079B55
:10AE0000626100F100403268606001F1004103F0CE
:10AE10000700E16022600DF5197DBDE8F08F0B9C05
:10AE2000034600F100400A46C4E90010DDE948018C
:10AE3000F5F772FABAF1000F02460B46AEDCBCE73A
:10AE4000089BDB00029372E4A29B022B06DC002B22
:10AE50000DDC7FF4A8AEA29A13469BE6A29B032BBF
:10AE60007FF4A1AE002348A91A46019106E700210C
:10AE7000084680E700231A4600E700BF0000704143
:10AE80000000703E000000002DE9F04F21F0004668
:10AE900087B0B6F1795F044601919046994604DA8D
:10AEA000F6F7AAFB002800F08F80019B2246194686
:10AEB0002046F5F7E9FB019B06460F463246194648
:10AEC00020463B46F5F7E0FB43A3D3E90023824647
:10AED0008B4630463946F5F7D7FB41A3D3E900232B
:10AEE000F5F71AFA32463B46F5F7CEFB3EA3D3E917
:10AEF0000023F5F713FA32463B46F5F7C5FB3CA3B2
:10AF0000D3E90023F5F708FA32463B46F5F7BCFBD8
:10AF100039A3D3E90023F5F701FA109BCDE902012B
:10AF2000002B37D0384B002240464946F5F7ACFBA2
:10AF3000DDE90223CDE9040150465946F5F7A4FBAB
:10AF400002460B46DDE90401F5F7E6F932463B46D9
:10AF5000F5F79AFB42464B46F5F7DEF928A3D3E90D
:10AF6000002306460F4650465946F5F78DFB02462C
:10AF70000B4630463946F5F7D1F902460B462046D6
:10AF80000199F5F7C9F904460D462046294607B050
:10AF9000BDE8F08F02460B4630463946F5F774FBA4
:10AFA00017A3D3E90023F5F7B7F952465B46F5F747
:10AFB0006BFB2246019BF5F7B1F904460D4620468E
:10AFC000294607B0BDE8F08F019D2046294607B00D
:10AFD000BDE8F08FAFF300807CD5CF5A3AD9E53D7C
:10AFE000EB9C2B8AE6E55A3E7DFEB157E31DC73E3A
:10AFF000D561C119A0012A3FA6F810111111813F96
:10B00000495555555555C53F0000E03F000000002B
:10B010002DE9F04FC64B83B021F000469E42044616
:10B0200001918A4611DDC34B9E4200F3B88000F0C7
:10B03000B380C14BC14AC24CBAF1000FD8BF13460E
:10B040002046194603B0BDE8F08FBE4B9E4200F388
:10B05000C180A3F1DE739E4240F3AE804FF0FF3B10
:10B06000019B224619462046F5F70EFB02460B4689
:10B0700080468946F5F708FB95A3D3E900230646E9
:10B080000F46F5F701FB94A3D3E90023F5F746F942
:10B0900032463B46F5F7F8FA91A3D3E90023F5F7DA
:10B0A0003DF932463B46F5F7EFFA8FA3D3E900238B
:10B0B000F5F734F932463B46F5F7E6FA8CA3D3E9C7
:10B0C0000023F5F72BF932463B46F5F7DDFA8AA364
:10B0D000D3E90023F5F722F942464B46F5F7D4FAB7
:10B0E00087A3D3E900238046894630463946F5F7E1
:10B0F000CBFA85A3D3E90023F5F70EF932463B4698
:10B10000F5F7C2FA82A3D3E90023F5F705F9324631
:10B110003B46F5F7B9FA80A3D3E90023F5F7FCF82D
:10B1200032463B46F5F7B0FA7DA3D3E90023F5F7A5
:10B13000F3F832463B46F5F7A7FABBF1FF3F02466C
:10B140000B466ED040464946F5F7E8F87E4E019B27
:10B150002246F5F799FA7D4B06EBCB064FEACB0B6F
:10B160009B44DBE90023F5F7D7F82246019BF5F76E
:10B17000D3F80B460246D6E90001F5F7CDF8BAF14F
:10B18000000F04460B46BFF65BAF01F100432046BB
:10B19000194603B0BDE8F08F00283FF44AAF019B89
:10B1A000224620461946F5F7B9F804460B462046D4
:10B1B000194603B0BDE8F08F5BA3D3E90023F5F790
:10B1C000ADF8634B0022F5F7EFFC00283FF446AFE3
:10B1D000534635E700F0C6F85E4B9E4204460D46E6
:10B1E00034DCA3F550239E4259DC02460B46F5F7AA
:10B1F00095F8574B0022F5F78FF8002206460F46C8
:10B2000020464FF080432946F5F788F802460B4662
:10B2100030463946F5F762FB4FF0000B04460191CA
:10B220001EE740464946F5F779F8019B2246F5F7B7
:10B230002BFA02460B4620460199F5F76DF80446B5
:10B240000B462046194603B0BDE8F08F424B9E42A4
:10B250001ADA424B0022F5F75FF8404B06460F46DC
:10B26000002220462946F5F70FFA394B0022F5F760
:10B2700055F802460B4630463946F5F72FFB4FF09E
:10B28000020B04460191EBE602460B4600203449CE
:10B29000F5F724FB4FF0030B04460191E0E62C4B3D
:10B2A0000022F5F739F82A4B06460F4620460022C1
:10B2B0002946F5F733F802460B4630463946F5F78E
:10B2C0000DFB4FF0010B04460191C9E6AFF300807E
:10B2D00011DA22E33AAD903FEB0D76244B7BA93F88
:10B2E000513DD0A0660DB13F6E204CC5CD45B73F56
:10B2F000FF8300922449C23F0D5555555555D53F02
:10B300002F6C6A2C44B4A2BF9AFDDE522DDEAD3FF5
:10B310006D9A74AFF2B0B33F711623FEC671BC3F95
:10B32000C4EB98999999C93F9C7500883CE4377E95
:10B33000FFFF0F440000F07FFB21F93FFB21F9BF25
:10B34000182D4454FFFFDB3F38BB000858BB0008F2
:10B350000000F03FFFFFF23F008003400000F83F95
:10B360000000F0BF21F00041704700BF0000000066
:10B37000F8B5C1F30A57A7F2FF35132D0B460C465B
:10B380000246064620DC002D40DB354F2F4101EA06
:10B39000070C5CEA000C14D02FA3D3E90023F4F7C8
:10B3A000BDFF00220023F5F7FFFB40B1002C03DABC
:10B3B0004FF480132B411C4424EA07040026324634
:10B3C000234610461946F8BD332D07DDB5F5806FCD
:10B3D000F7D1F4F7A3FF02460B46F2E7A7F21347B3
:10B3E0004FF0FF3C2CFA07F70742EAD01AA3D3E943
:10B3F0000023F4F793FF00220023F5F7D5FB002884
:10B40000DDD0002C1BDB26EA0706D8E712A3D3E920
:10B410000023F4F783FF00220023F5F7C5FB002883
:10B42000CDD0002C02DB00263446C8E724F00043D0
:10B430000C4A1E43002E18BF14460026BFE7142DE9
:10B4400008D00122C5F1340302FA03F39E1928BF84
:10B45000A418D8E70134D6E79C7500883CE4377E11
:10B46000FFFF0F000000F0BF01490020704700BF40
:10B470000000F87F00000000F8B5C1F30A5304464D
:10B480000D460E46174673BB21F000460346334374
:10B4900028D0314B0022F5F7F7F8304B9F42044695
:10B4A0000D461ADBC1F30A530E46363B3B4440F2CD
:10B4B000FE72934220DC002B3CDC13F1350F2CDABA
:10B4C0004CF250339F4217DC05F0004343F0D27139
:10B4D00041F4B731224841F01F011BA3D3E90023F7
:10B4E000F5F7D2F8F8BD40F2FF729342DED1024682
:10B4F0000B46F4F713FFF8BD05F0004343F0FC41A1
:10B5000041F45F1141F4105111A3D3E90023154810
:10B5100041F03C01F5F7B8F8F8BD26F0FF4626F4F7
:10B52000E006363346EA035120460F4B0022F5F77A
:10B53000ABF8F8BD26F0FF4626F4E006204646EAC2
:10B540000351F8BDAFF3008059F3F8C21F6EA50197
:10B550009C7500883CE4377E00005043B03CFFFF00
:10B5600059F3F8C29C7500880000903CF8B500BF04
:10B57000F8BC08BC9E467047F8B500BFF8BC08BCD4
:04B580009E4670472C
:10B5880000000000000000000000000000000000B3
:10B59800000000000100000002000000030000009D
:10B5A800040000000000000005000000000000008A
:10B5B800000000000000000006000000000000007D
:10B5C800000000000000000007000000000000006C
:10B5D8000102030401020304060708090006101605
:10B5E800000610160001020304050607080C1014D3
:10B5F80018203040010002000400060008000A007C
:10B608000C00100020004000800000010804020423
:10B61800080101010101010307010000005EBCE20D
:10B62800613FDD83C29C7E20A3FD1F419DC3217F16
:10B63800FCA2401E5F01E3BD3E6082DC237D9FC10A
:10B64800421CFEA0E1BF5D0380DE3C62BEE0025CFE
:10B65800DF81633D7C22C09E1D43A1FF4618FAA4EA
:10B6680027799BC584DA3866E5BB5907DB856739D6
:10B67800BAE406581947A5FB7826C49A653BD987CA
:10B68800045AB8E6A7F91B45C6987A24F8A6441ABE
:10B6980099C7257B3A6486D85B05E7B98CD2306EAA
:10B6A800EDB3510F4E10F2AC2F7193CD114FADF396
:10B6B800702ECC92D38D6F31B2EC0E50AFF1134D8A
:10B6C800CE90722C6D33D18F0C52B0EE326C8ED07E
:10B6D800530DEFB1F0AE4C1291CF2D73CA9476286A
:10B6E800ABF517490856B4EA6937D58B5709EBB556
:10B6F80036688AD495CB2977F4AA4816E9B7550B4A
:10B7080088D6346A2B7597C94A14F6A8742AC8963D
:10B71800154BA9F7B6E80A54D7896B35000089118B
:10B7280012239B322446AD573665BF74488CC19DA1
:10B738005AAFD3BE6CCAE5DB7EE9F7F88110080181
:10B7480093331A22A5562C47B7753E64C99C408D81
:10B75800DBBF52AEEDDA64CBFFF976E802218B301D
:10B76800100299132667AF763444BD554AADC3BC61
:10B77800588ED19F6EEBE7FA7CC8F5D983310A2041
:10B7880091121803A7772E66B5543C45CBBD42AC41
:10B79800D99E508FEFFB66EAFDD874C904428D53D9
:10B7A80016619F702004A9153227BB364CCEC5DF21
:10B7B8005EEDD7FC6888E1997AABF3BA85520C4301
:10B7C80097711E60A1142805B3373A26CDDE44CF01
:10B7D800DFFD56ECE9986089FBBB72AA06638F729D
:10B7E80014409D512225AB343006B9174EEFC7FEE1
:10B7F8005CCCD5DD6AA9E3B8788AF19B87730E62C1
:10B8080095501C41A3352A24B1163807CFFF46EEC0
:10B81800DDDC54CDEBB962A8F99A708B0884819568
:10B828001AA793B62CC2A5D33EE1B7F04008C919B0
:10B83800522BDB3A644EED5F766DFF7C8994008570
:10B848009BB712A6ADD224C3BFF136E0C118480990
:10B85800D33B5A2AE55E6C4FF77D7E6C0AA583B40C
:10B86800188691972EE3A7F23CC0B5D14229CB3870
:10B87800500AD91B666FEF7E744CFD5D8BB502A430
:10B8880099961087AFF326E2BDD034C1C3394A2850
:10B89800D11A580BE77F6E6EF55C7C4D0CC685D7C8
:10B8A8001EE597F42880A1913AA3B3B2444ACD5B30
:10B8B8005669DF78600CE91D722FFB3E8DD604C7F0
:10B8C8009FF516E4A9902081BBB332A2C55A4C4B10
:10B8D800D7795E68E11C680DF33F7A2E0EE787F68C
:10B8E8001CC495D52AA1A3B03882B193466BCF7AF0
:10B8F8005448DD59622DEB3C700EF91F8FF706E6B0
:10B908009DD414C5ABB122A0B9923083C77B4E6ACF
:10B91800D5585C49E33D6A2CF11E780F28000024B5
:10B928000000000000000000182D4454FB21E9BF6E
:10B93800D221337F7CD90240D221337F7CD902C007
:10B948000000000000000080182D4454FB2109402D
:10B95800182D4454FB2109C0FB21F93FFB21094064
:10B968007CD91240FB2119407A6A1F407CD92240B9
:10B97800BBFD2540FB2129403A462C407A6A2F40DE
:10B988005C4731407CD932409C6B3440BBFD35402C
:10B99800DB8F3740FB2139401BB43A403A463C40E4
:10B9A8005AD83D407A6A3F404C7E40405C4741400F
:10B9B8006C1042407CD942408CA243409C6B44406E
:10B9C800AC344540BBFD4540CBC64640DB8F4740C5
:10B9D800EB584840FB21494083F9A200444E6E00D1
:10B9E800FC291500D1572700DD34F50062DBC000C3
:10B9F8003C999500419043006351FE00BBDEAB00CB
:10BA0800B761C5003A6E2400D24D42004906E000F5
:10BA180009EA2E001C92D100EB1DFE0029B11C0082
:10BA2800E83EA700F535820044BB2E009CE984005F
:10BA3800B4267000417E5F00D691390053833900E7
:10BA48009CF439008B5F840028F9BD00F81F3B0087
:10BA5800DEFF97000F980500112FEF000A5A8B00A0
:10BA68006D1F6D00CF7E360009CB2700464FB7000B
:10BA78009E663F002DEA5F00BA277500E5EBC70018
:10BA88003D7BF100F739070092528A00FB6BEA0010
:10BA98001FB15F00085D8D00300356007BFC460037
:10BAA800F0AB6B0020BCCF0036F49A00E3A91D0070
:10BAB8005E619100081BE60085996500A0145F008F
:10BAC8008D40680080D8FF0027734D0006063100BE
:10BAD800CA561500C9A873007BE260006B8CC000D1
:10BAE80000000040FB21F93F000000002D44743E97
:10BAF800000000809846F83C0000006051CC783B7C
:10BB080000000080831BF0390000004020257A38AF
:10BB1800000000802282E336000000001DF3693532
:10BB280002000000030000000400000006000000FE
:10BB38004FBB610567ACDD3F182D4454FB21E93F3D
:10BB48009BF681D20B73EF3F182D4454FB21F93F2C
:10BB5800E2652F227F2B7A3C075C143326A6813CB2
:10BB6800BDCBF07A8807703C075C143326A6913C5D
:08BB78005C56FF7F0100000094
:08BB8000F58F0008F502000832
:04BB8800D1020008DE
:10BB8C000090D0030090D0030100000010000000D2
:10BB9C0066666666666606C0000000000000E0BFD0
:10BBAC002800002400000000000000001403002402
:10BBBC007C030024E40300240000000000000000CB
:10BBCC000000000000000000000000000000000069
:10BBDC000000000000000000000000000000000059
:10BBEC000000000000000000000000000000000049
:10BBFC000000000000000000000000000000000039
:10BC0C000000000000000000000000000000000028
:10BC1C000000000000000000000000000000000018
:10BC2C000000000000000000000000000000000008
:10BC3C0000000000000000000000000000000000F8
:10BC4C0000000000000000000000000000000000E8
:10BC5C0001000000000000000E33CDAB34126DE685
:10BC6C00ECDE05000B0000000000000000000000EE
:10BC7C0000000000000000000000000000000000B8
:10BC8C0000000000000000000000000000000000A8
:10BC9C000000000000000000000000000000000098
:10BCAC000000000000000000000000000000000088
:08BFDC00CC150024FF00000059
:04000005080020E5EA
:00000001FF
